:400000000010002011000000650400006504000010B50C4A0C4B1A600C4B1A68102313400B4A00D113601368802B09D10023136000F096F8002803D000F092F800F0A8F8B0
:4000400001F040F96588EDAC38000340540003406000002000000000000000000000000000000000000000000000000000000000000000000000000000000000000000003E
:400080000000000000000000000000000000000000000000000000000000000000000000000000000000000000000000000000000000000000000000000000000000000040
:4000C00000000000000000000000000000000000000000000000000000000000000000004C0A003561700000BB11072B0000000000000000000000000000000000000000A6
:4001000010B5064C2378002B07D1054B002B02D0044800E000BF0123237010BD0001002000000000CC130000084B10B5002B03D00749084800E000BF07480368002B00D143
:4001400010BD064B002BFBD09847F9E70000000004010020CC1300006800002000000000074B1A78074B1878074B000219780B04184303001343054A1078000618437047C3
:40018000C1FF0000C2FF0000C3FF0000C4FF00000047000070B51D491D4BCC58002C34D00C3BCC5063052BD5C86D1A4BCA6D40041A600022400F824208DA15001835AD002B
:4001C0004E59013295005E51D2B2F4E707200F211A68550A05401140012902D1120B02420ED05A1CD27F002A03D09A1CD27F954206D001215A1CD1779A1CD57740225A6200
:40020000A30502D50122034B5A6270BD00000A400C05000080010020031E0CD00023994209D04118814204D0027801309B18DBB2F8E75B42DBB2180070470000F8B50400B1
:40024000A37A407AE17A1B02034309041A000B00217B1343090619430626002935D0A57963792D021D43ED012800194F803043189C46BB4229D8A278637812021A43E3784D
:400280001B041A4323791B06134398421DD89C451BD9FFF7C1FF2378834216D12C008134FF34BC4211D80B4B22889A420DD12800E179A379090219438B300A39FF30FFF731
:4002C000ABFF237A834200D100263000F8BDC046FFFF000059430000182310B5584301F017F810BDF8B5D02580221E4C1E4BED00635163591D4F1E4E3B406351A359920005
:400300001343A3511420FFF7E7FFA0228021D2000905A1506359E0201F40164B675163510125400023582B432350C923A058084203D1013B9BB2002BF8D10220FFF7CCFF23
:40034000E0235B00E0588022A0231205DB00E250A259094B000C1340A351084BC0B25843400AF8BD00000A4000020080FFFFF7FFCC08000000020200FFFDFFFF50C30000B8
:4003800010B5FFF7AFFF064B984203D96420FFF7A3FFF6E780230349034A9B01D15010BD821400002000040000000A4070B5802504002D02AC4205D9054800F0A9FF054B0C
:4003C000E418F7E70448604300F0A2FF70BDC0460000E02E0080FFFFC05D0000F8B5070001200E001500FFF7E1FF174C4020230028331B782A03384310435B021843134B14
:40040000134AD8601278D9685001802252000A430243DA600022AA4206D291007058111D890058500132F6E780210A4A8902136803200B431360FFF7B9FF072228342378F0
:40044000013313402370F8BD8001002000000A406C000020C4000A40002210B51100FFF7BDFF10BD10B500F063FF03680C2B00D1FEE7FEE7002370B539483A4C3A4D9A00ED
:400480002100032B00D8A95801338150172BF6D172B6CC22354B12041A60354A354B07251A601222344B354C1A6000F03AFF2368334AAB432360334B33491B780600DBB2CB
:4004C0001360324A1368AB431360314B0A6818787F239A43034013430B60322000F018FF052223683220AB431343236000F010FF062223683000AB431343236000F015FF5F
:40050000244A254B25491A60254B264A1A609E22D2010A602449196024490A60BC21244A89011A60234A1160C021234A89001A60224A11608021224A49001A60214A1160DA
:40054000214A1A604022214B1A60214B1A68002A00D11A6001211F4A13680B43136070BD00000020650400000000000000000240306003000800044030001040080F034073
:400580000C0F0340FDF1FF0F180F0340100F0340E4F1FF0F007F070000030140100201400000014040FF008004FF00800C02014003FF00800802014002FF008004020140AE
:4005C00001FF00800002014000FF0080280003406000002000001040F0B5C74CC74DC84A6359C84E134363510423F361023B3361002373624033F3622368C1225B005B088C
:400600002360802309211B062360D200A358ADB08B4308390B43A3508832A35827008B40CB40A350A35817310B43A3506259B64B13401222134363516259B44B1340AA22FD
:40064000920313436351FFF74DFEAD4AB04B01950290079203960025984206D8FFF742FEAC4B02909842F9D901250124FFF73AFE029BC833984201D300240290029B1B1ABF
:40068000C72B01D90134E4B2002D5CD0A24B984259D80221A14AA24E1368A2488B431360936836318B4308390B4393603368C0318B4350390B4333603C589B499B4D214077
:4006C0000324214339509A489A49053478509A48894B39582143395018383958974C89B2214339507959964801430F20795195490C688443E1B2944C2468059224090440F3
:400700000C4306960295914A914E924D92499348112C1ED09C5834408026B60026439E503C269C58B4431C3E34439C50029C1C5925408024A4022543029C1D515C5820404E
:40074000E024E4031AE00A20FFF7C6FD0A2C8DD99FE79C5834408026760034439C509C58C43EB4432C3E34439C50029C1C592540029C1D515C582040C024A40320435850C0
:40078000C020F8247B588002034375487B503B58640323433B501F201825724C724E236883432B432360714C113D23688343033803436F4823603C586E4B2340F824E4022A
:4007C0002343FF243B503B58A3432B433B506A483B58A343F03C23433B503C58674B2340A024640223433B506548664B3C582340F024240323433B50C6207B5801241B0BE2
:400800001B0303437B50604960487B585B0D5B0503437B505E495F487B585B0B5B03034380207B505C4940057B581B011B09034380207B507B58000503437B50BB586420C8
:40084000A343BB508022BB5912061343BB51FFF743FD1222019BA820FB5850491343019AC000BB5000224E4BFC504E4BFA50019B4D4AFB589B025B0EBB508023DB053B5052
:400880007A5814437C503C581B4A1C42FBD0019B464CD058464B250003400198313513508020A823C005DB00D05001205358834353501A21019B3F48D3588B43019953507C
:4008C00000232B70FFF7BAFC002801D004232B702300082131331A7837480A4337491A700A68049192B282426AD100220A6001211A780A431A706BE000000A40F4080000C9
:4009000004000010FC0001400700C0FFFF7FC0FF9F0F000081140000931100000000044000000240DC080000FFFFFF1BD408000048600000E4080000F808000000000F0477
:400940007F100000E80F00F0EC0F00F0942000003FFCFFFFFF3FFCFFD8080000FFFF0FFF2820000084FF0A406420000088FF0A40A0200000FF3FC0FFA4200000FF3FF0FFEC
:40098000A8200000FF0FE0FF88200000FF0400008C200000FA04000090200000502000004C2000005C20000058200000800100201F00C0FFC0FF00004C4200006000002061
:4009C000049A12681A780423134001D100F003FC3022DB4B01265A80DA4A09209A80DA80D13AFF3A1A81019B079AFB5890251A431300019A2D01BB500322039B9E60039B11
:400A0000DA6004230399CB610399023B0B610021039B596240230399CB623B68C121B340F3403B6080231B063B60C9007B58834333437B507B595B301A437A51FFF74CFC95
:400A4000D223DB00FA581821B240F240FA50FA580A43FA507A5910390A437A512531BA4AFF311160B949BA4A1160C021C9007A58B240F2407A50FA58B240F240FA50B54AF5
:400A80002033FA507B58B44A1343C2227B501421D200BB588B43BB50B04B0D311A68FF310A4300211A60AE4A1160AE49AE4A11608E211A68FF3116431E60AC4AAC4B1A6095
:400AC000AC4A13685B0A5B020B4313602023AA4AAA491360AA4A1160AA4AAB491360A023A122DB00F950D200BB580B43BB5062B6220032321578002D4FD1C026F600002346
:400B000008AAD3719D4203D1BA59A04B134003E08822BB5952001343BB510A20FFF7DCFBAD239B00FA58A0235B01134080225201934202D1012308AAD37108ABDA79AB00D8
:400B4000D2B2002A23D0E218516B01315163516B8F4A91421DD90022A11CEDB2E5636263A263CA77210028310A70611CCA772200012132321170C0220420D200B958814381
:400B8000B950B9580B43BB50FFF7FAFB24E0E3185A630135022D1FD0B1E7AD239B00F9584D33FF331940E36B9B00E318002912D0596B01315963E36B9B00E318596B744B60
:400BC000994209D980210023724889016363A3634350137000E05963666A012E21D1002500F09FFB656200F0A0FBA31CDD77230028331D70631CDD7780239B01FD50F2252C
:400C00009620ED007B59400033437B51FFF7CEFB7B59B3437B51FFF7B3FB230032331E70A8E2636A402B00D0A4E200F07AFB0023636200F07AFB0F2325682B406D046D0FCB
:400C400000D14FE2022B0DD10320FFF705FC3220FFF7ACFB0620FFF7FFFB2300032232331A7087E20F2B00D084E2354B1A78012A00D13DE76279D20925D02079C006C00E2E
:400C80000138032800D975E200F07EFB020E121A414B21002364414B403163640023A3643F4B0422E36419E23E4B23643E4B02E03E4B2364012321006364403102220DE2CC
:400CC0003B4B236407E2E2883A498A4200D0F4E1210026792000F206D20E0192354A603102914A8018216130027876098A4310390A4302701F20029972010978013D0840FC
:400D0000029902430A70019AAD00501EEDB20C2800D9D2E100F042FB0D0050007A00AC00D101CE00E100FB0062017E019F01A801B201002D42D12F236566A366032291E23C
:400D40006C000020FF010000D0000A400A404101D4000A4061643D008A0E304FC4000A40A8000A400B410000BC000A400F020000B4000A40E4000A4080E100E095010000A4
:400D80005400002000E100E003060100EFFEFFFFC409000000000A40418000FFB4040092000060F6428000FF0000B4044380B4044480B404B4040000002D09D02200182109
:400DC000613213788B4308390B431370012249E22200E023643203CB03C22300210031331B7829315B0707D4C64B5B681902090CC90161310293FF31200008226C3000F08C
:400E0000D7FA002307226367A3672BE2042DD5D1237A532BD2D1BC4B00209B6CA366BB4B1A78BB4BD1B2E1661B781B020B431A00E366B84B1B781B041343B74AE366127840
:400E400012061343E366B54B1A78B54BD1B221671B781B020B431A002367B24B1B781B041343B14A2367127812061343236706E2042DA3D1237A522BA0D172B6049B049AF3
:400E80001B68F225136080230022012696209B01FA50ED007B59400033437B51FFF786FA7B59A24AB3437B511368A1499BB20B4313605FE1042D81D12300227A7C33502A44
:400EC00007D118784E3A904300D0D6E11A70033DD5E1002001251870D1E1701EC3B2052B00D96BE718235843C0B2062E03D09D4200D063E702E0082D00D05FE721008D4BDC
:400F00000830181808312A0000F052FA32E1042D00D053E7884A127A002A00D04EE7227A462A00D04AE7A27A0E201102627A0A43160022007C321278002A45D05A8807386C
:400F4000B24241D89A88B24202D2DB88B3423BD17A4B07209E4237D83022794D7549AB6A08319343203A1343AB6270320CA800F01FFA744B74490A937F230B930AAB8B602C
:400F8000724B4B60C046C046C0468B681B0F1A070A2B10D16E48330403430A930AAB8B606C4B4B60C046C046C0468B6800211B0F1B07934200D00C213022AB6A0800934308
:400FC000AB62002900D005205C4B9E4267D122000421313213780B43137060E0002D00D0ECE6711ECBB2052B00D9E7E6182359430822C9B2062E00D01A0020004D4B083185
:401000006430591800F0D4F90722062E00D029E1043A27E1042D00D0D0E6227A462A00D0CCE6A17A627A0902114322007C3212780E20002A33D01B8907388B422FD23F4BE6
:4010400099422CD881403B4880220830033D00F0AFF9280013E1042D00D0AFE6267A012E00D1EDE007201AE0002D00D0A6E6230031331A78230060331A710EE0082D00D085
:401080009CE6A068E168344B42189A4200D995E6FFF7C2F82300603318710222E2E022001F210125603213788B4301990B43137001350230EAB26066DCE062682749130CC2
:4010C0008B4257D1E723110A22640B402200102141320B4313702100012240310F20FFF77DF947E0092B45D1230032331878032840D11B4E3378002B34D10130FFF7ACF949
:4011000038E0C046C0FF0000FCF0FF0F78F1FF0F79F1FF0F7AF1FF0F7BF1FF0F7CF1FF0F7DF1FF0F7EF1FF0F7FF1FF0F0CED00E00400FA050002002080020020FF01000064
:4011400000000340B6D700000000104004000080B6D8000005000080FFFF0000B40400006C000020FFF778F92021494A13688B4313603570210032310A78012A13D1202580
:40118000434803682B430360424B1A7002230B700021414B414A99504149424A99500521414A9950A4E4022A00D0A1E43A4D3E4EAB59DB0300D49BE43649013A10000C319F
:4011C000FFF70CF90022354BEA50364B344AEA500523AB518CE4354A354953720222059B1B689343059A13603822059B9B689343083A1343059A9360F022069B1B68934351
:40120000069A136080220B68120613430B60BB5928495B005B08BB51019BFB581343019ABB50029BFA58244B1340029ABB508023049A1360214A13689BB20B43136057E438
:401240001F48FEF7FBFF21003131002804D10B78AB430B70350012E00A78062015430D7035000CE021001F2060310B788343019803430B702100603130E70125032022001F
:401280001F21603213788B4301990B4313700FE7C4000A406C000020001000E018D00000FFEA410014D0000010D0000080020020DC000A400400FA0580EFFFFF0CED00E031
:4012C000C0FF0000F8B500250E490F4B01394A1C14D000221F685C689E68A018B24203D0B858A0500432F8E70200DE68141AA64201D020C2FAE710330139E8E700F01EF8DD
:40130000FFF76AF901000000F8130000000000000230800803D00138FDD1C046C046C0467047EFF3108072B6704780F310887047014B18687047C046E00000200E4B70B5D1
:4013400000251E000D4CE41AA410A54204D0AB00F35898470135F8E700F03CF8084B00251E00084CE41AA410A54204D0AB00F35898470135F8E770BDE0130000E013000002
:40138000E0130000E813000002B4714649084900095C49008E4402BC7047C04603B47146490840004900095A49008E4403BC7047002310B59A4203D0CC5CC4540133F9E716
:4013C00010BD000027000000001500000000000043000000F8B5C046F8BC08BC9E4670472901000075040000F8B5C046F8BC08BC9E467047010100000814000068000020CC
:4014000080000000A8010000000000000100000200020002000200005A90010A32000000000000000000000000000000000000000000000000000000000000000000000053
:40144000D013000000000000000000000000000000000000000000000000000000000000000000000000000000000000000000000000000000000000000000000000000089
:40148000800000200000000000000000000000000000000000000000000000000000000000000000000000000000000000000000000000000000000000000000000000008C
:4014C00000000000000000000000000000000000000000000000000000000000000000000000000000000000000000000000000000000000000000000000000000000000EC
:4015000000000000000000000000000000000000000000000000000000000000000000000000000000000000000000000000000000000000000000000000000000000000AB
:40154000000000000000000000000000000000000000000000000000000000000000000000000000000000000000000000000000000000000000000000000000000000006B
:40158000000000000000000000000000000000000000000000000000000000000000000000000000000000000000000000000000000000000000000000000000000000002B
:4015C00000000000000000000000000000000000000000000000000000000000000000000000000000000000000000000000000000000000000000000000000000000000EB
:4016000000000000000000000000000000000000000000000000000000000000000000000000000000000000000000000000000000000000000000000000000000000000AA
:40164000000000000000000000000000000000000000000000000000000000000000000000000000000000000000000000000000000000000000000000000000000000006A
:40168000000000000000000000000000000000000000000000000000000000000000000000000000000000000000000000000000000000000000000000000000000000002A
:4016C00000000000000000000000000000000000000000000000000000000000000000000000000000000000000000000000000000000000000000000000000000000000EA
:4017000000000000000000000000000000000000000000000000000000000000000000000000000000000000000000000000000000000000000000000000000000000000A9
:401740000000000000000000000000000000000000000000000000000000000000000000000000000000000000000000000000000000000000000000000000000000000069
:401780000000000000000000000000000000000000000000000000000000000000000000000000000000000000000000000000000000000000000000000000000000000029
:4017C00000000000000000000000000000000000000000000000000000000000000000000000000000000000000000000000000000000000000000000000000000000000E9
:4018000000100020011D00005568000055680000000000000000000000000000000000000000000000000000000000000000000000000000000000000000000000000000E0
:401840000000000000000000000000000000000000000000000000000000000000000000000000000000000000000000000000000000000000000000000000000000000068
:401880000000000000000000000000000000000000000000000000000000000000000000000000000000000000000000000000000000000000000000000000000000000028
:4018C0000000000000000000000000000000000000000000000000000000000000000000590A003561700000BB11072B000000000000000000000000000000000000000081
:401900005943000F012000041330B4040100010000020B000000000000000000000000000C021800240200002402000024021800000000000000000000000000000000001D
:40194000010102000000001C0006BF0000070100000001000000000000000000000000002C9101032CD102002CB10400E14006003C2140C92D21A4C9000000000000000090
:40198000000000000000000000000000000000000000000000000000000000000000000000000000000000002F003C02400248024C020000500260029C020000000000008E
:4019C00000000000000000000000000000000000000000000000000000000000000000000000000000000000000000000000000000000000000000000000000000000000E7
:401A000000000000000000000000000000000000000000000000000000000000000000000000000000000000000000000000000000000000000000000000000000000000A6
:401A40000000000000000000000000000000000000000000000000000000000000000000000000000000000000000000000000000000000000000000000000000000000066
:401A80000000000000000000000000000000000000000000000000000000000000000000000000000000000000000000000000000000000000000000000000000000000026
:401AC00000000000000000000000000000000000000000000000000000000000000000000000000000000000000000000000000000000000000000000000000000000000E6
:401B0000B4046DF643797072657373001800000041A000FFB40480010000000000006DF600000000B4046DF6000000000101000000020000000000000001002D04140A029C
:401B400008140A020000000004460A02040004021000DD018D030A0000000000000000003C03100E204E8813400D030018F6000000000000320000001400C8000501020279
:401B800018010000020FC80F16000000000000000000000016001400C8000000181F0000020200030F49720000000000000000000000000000000000000000000000000014
:401BC00000000000000000000000000000000000000000000000000000000000000000000000000000000000000000000000000000000000000000000000000000000000E5
:401C000000000000000000000000000000000000000000000000000000000000000000000000000000000000000000000000000000000000000000000000000000000000A4
:401C40000000000000000000000000000000000000000000000000000000000000000000000000000000000000000000000000000000000000000000000000000000000064
:401C80000000000000000000000000000000000000000000000000000000000000000000000000000000000000000000000000000000000000000000000000000000000024
:401CC00000000000000000000000000000000000000000000000000000000000000000000000000000000000000000000000000000000000000000000000000000000000E4
:401D000010B5044B83F30888034A044B1A6005F029FBC046001000206588EDAC3800034010B5064C2378002B07D1054B002B02D0044800E000BF0123237010BD0001002091
:401D40000000000040F30000084B10B5002B03D00749084800E000BF07480368002B00D110BD064B002BFBD09847F9E7000000000401002040F30000680000200000000072
:401D80007047704770B570244443064E0500A359002B02D098470023A3510122024B5A5570BDC04688040020F8040020704700000122014B1A707047E402002010B50CF0E5
:401DC000CDFD002010BD00007023434310B5044AD3184B331B78002B01D00DF07BF810BD8804002070B52F4C2388632B01D86423238063882288934208D99B1A9BB21D1CBD
:401E0000042B00D904255519ADB207E0D31A9BB21D1C042B00D90425521B95B201262900002005F021F8204B25801E606388AB4235D040251D4B1E4A1D601E4B9A650CF066
:401E4000A0FCC0231C4A1B0411680B4313600CF09CFC1A4B1D602379002B0ED18121184A890411600C21174A1160174ABC311660164A1160164A136026710CF082FC01216C
:401E8000144A13680B4313600CF07FFC0CF079FC8022114B52041A600CF077FC01E004F07FFD70BD1C0100203001094080E100E0E51D00000000002004E400E000E100E042
:401EC0000001094024010940380109401401094008010940000009400800094070B5040015000CF0D7FD70236343074A0321D318002800D004211973702161430831511837
:401F00002000A84770BDC0468804002010B50BF04DFF10BDF7B50C000092050003F032F8B8235B006B43224F0098FB18FE33604364211E8B0DF0C6F80019C343DB17184048
:401F40001C4B400019780DF0BDF8B6B280B2000231000DF02DF80400032803D9FE2802D9FE2400E004240CF00CFCB8235B006B43FF18FF377B7D0190002B02D080231B03D6
:401F80001C43D0260C4FF600BB590A2000930B4B1C43BC5104F0EDFB28000099BC5904F00BFE01980CF0F1FB0120E40BA043FEBD040300208800002000000A4000020200ED
:401FC00010B5040001210CF00DFF022120000CF009FF012010BD000010B504000CF0BEFC763002780C4B002A03D11A195279012A03D10A4A125D002A03D01A199279002AA0
:4020000009D0002201211B199A71044B2000195503310CF01BFD10BD1C010020E502002010B50400042905D1074B1B18D9790CF021FF08E0032906D10CF090FC024B9C30C3
:402040001C190378E37110BD1C010020F8B570244443184B05001C194B342378002B27D00CF08FFB01216027134B144E9A598A439A51B53EFF3E9A593A439A51104E9A593B
:402080008A4310499A515E580F4A324084265A500E495A58B2435A500CF077FB2800002500210CF0B9FE257004F07AFC084B1D80F8BDC0468804002000000A40F408000067
:4020C000442000003020000010C0FFFFF80800001C010020F0235843034BC01898300088024BC0187047C0462019000000190000F0235843034BC01896300088024BC01882
:402100007047C0462019000000190000F022044B50435B5CC018034B185A034BC018704744F30000201900000019000070B50400FFF7DEFF70236343354A0600D318C82258
:402140001D8E9200954201D1324A1A8620000CF005FC5C233F22FF33C35C9343C02B01D0738AED182C4B1B5D002B03D02B4B6200D35AED182A4EB5420ED8002C47D12000CB
:40218000572106F0D5FEC823A8B29B009D420AD8200007F08FFB3AE0002C38D12000572106F0C6FE300014210CF002FF14231D4D58432A881C4B84B29A4204D80022013300
:4021C0002B801A4B1A801A4E3378052B0BD0002004F01CFD04F0C2FF144B1880142358430C4BC01828800020124B1C80124B18702B88A34207D104230122337057210F4B68
:4022000006F0BAFE03E05721307007F0CFF870BD88040020881300007C04002080040020FC530000A00600201F030000A6060020F00200209E060020A2060020AD9300009E
:40224000F7B50E0004000CF089FB702301216343644A654DD318654A00901E86AB588B43AB50634B1B78002B18D1624A624BA958624F0B4002210B43AB50614B38001B783D
:4022800007F05AF85F4B188004F076FF01225E4B1F80574B1A7005225C4B1A705C4B1F5D002F14D12000FFF723FF038A002B0ED001231421564A1355564A63009952564A47
:4022C00056499F52564AA3009950564B1F553100200003F027F80CF054FA012252496B5893436B50514BEA50B8235B006343504AD3180022FC335A660CF047FA20000CF0AD
:402300002DFB5C223F21FF32835C364F8B4301922000C02B3FD103F09BF820000CF01EFB0300FC33DA6C9B6C9A4236D0A22305225B00C35C64255B065B0E5343632B00DDB0
:402340001D00019BC35C1B070DD58423FF33C05C384B584370236343FB18198E0CF028FE854200D9050070236343FB184B331A78314B002A03D05D80FFF734FD04E02900CE
:4023800020001D8004F070FD702301226343FB184B331A7001E0FFF759FE200005F042FB70236343FF18C823398E7A8E9B00914205D39E4211D0200005F060FA0DE09E42BB
:4023C0000BD0009B72331B78002B06D045373B78002B02D0200005F003FA2000FFF7A6FEF7BDC0468804002000000A40EC080000AB060020F40800000700C0FF8813000064
:40240000A6F2FF0FA6060020A0060020F00200207C0400207E04002080040020811D000084040020F8040020442000003C20000004030020A08601001C01002070B5041E78
:402440003ED1204B1A78012A3AD001221E4D1A702B78934203D11D2106F06AFD2C70F2231A49DB00CA581F239208194D1A4019482A7008580026800818401300164C5B0836
:402480000136002B01D0F6B2F9E70121B1400600C9B2297076080133002E01D0DBB2F9E701369E40F3B2237049088A4200D12A705B08984200D120701D21002003F0E6FF6D
:4024C00070BDC0466F0600206C06002000000A406D060020940700006E06002070B5002827D1144B1A78012A23D00122124C1A702378934202D11D2106F01AFDF2231F2233
:402500000E49DB00CB580E489B0813400D4D0370495989080A400C490A702278002A02D15B08037001E0002323701D21002003F0ADFF70BD6C0600206F06002000000A4042
:402540006D060020940700006E06002070B570244443244B05001C1945342378002B3FD10BF076FCFA22204B5200C3189BB2934213D91E4B984202D92800FFF7AFFF1C4CE0
:40258000642223005E21280006F0F6FC230001225D21280006F0F0FC22E001232370002D1ED190250A2004F0E4F80322114C2D01635932201343635104F0DBF8082263591C
:4025C00032201343635104F0D4F8802302219B01E2580A43E250E2588A43E250064AE25070BDC0468804002072EDFFFF82140000A52D000000000A4020000400F0B58FB0F3
:402600000E00040017000CF093FA0500701E392800D9D8E10CF08AFE790062007900C700C700D701D701D701D70179006C00D701D701D701D701D7015F026E00D701CF0108
:402640006E00DA00D701D701D7017900D701D701D701FC00D701D7012A01D7013A00D701D701D701D701CA01D701D701D701D7015F02D701C301D701D701D701D701D701E0
:40268000D7015F02D701D7016E00D6005A21200006F034FCD54F002803D03B199B79002B0AD15A21200006F043FCFA22D04B92005A21200006F060FC6F353B192A781B7AEA
:4026C0009A4207D0092210006043CA4B0021C0180CF019FE2B783F193B72FCE170236343C54AD318190000223A310A70393368E1012700E0002776352B780125002B06D0F7
:402700003500153D6B425D4101E000252F0070236343B94A0021D318180039333A30017019700192032E01D01A2E14D15A21200006F0E4FB002804D0AC4B1B199B79002BCA
:4027400003D15A21200006F0F3FB0022AB4B1A55A64B1B195A71002F05D1002D03D12921200006F0E5FB012E0FD1092300226343A349A0485918C318985C8D5C854200D2B0
:402780007CE10132092AF7D16CE1032E02D01A2E00D018E1F02280209A49D2008B58000603438B500FE170236343934A0121D3181A003A32117019000022393144330A700C
:4027C0001A7000E1894B01221B191FE0702394352A7889496343012A03D9CB183B33012202E00022CB183B331A7002223B799343012B00D06FE15A21200006F099FB7B4B8F
:402800001B199A79002A00D165E100229A7162E1FB79B978DA091DD01A205B061B0F01335843FA88D205D20D824213D903AA5170002151800F310B40DB0075310B43387845
:40284000D3706A4B10700C3393601B23773913736D4B07E002239943092900D13BE1002312211A0020000CF093F834E10BF089FF664B01901B78002B00D18CE0614D644F2E
:402880003721200006F054FBEA59624B5520134002221343EB51404204F06EFCEB590A205B005B08EB5103F064FF5B4A5B49AB585B4F0B43AB500222EB5932201343EB51C4
:4028C00003F057FF574A584BA95801200B400F210B43AB5003F04DFFFF21544A544B2000EA50544BEA588A43EA50EA588A43FD390A43EA50E958504A0A40EA50FFF7F8FB73
:40290000437F002B0DD00230C37F002B09D080228021EB59C9049343484AEB51AB580B43AB5080218027464A0905AB5801200B43AB50444A0A2113683F065B005B08136014
:402940000023062206F04CFC3F4A2000AB583B43AB500BF0C7FC44213C4AAB588B43AB50FA230122DB00E9589143E950E9580F43FC21EF5089006B5893436B50FA239B0047
:40298000EA500022324B70391A606858314B03406B501E4B1A7001980BF0F7FE9BE070236343154AD3183A3300220AE001220F4B1B195A718FE0702363430F4AD318012263
:4029C00049331A7087E0172E00D17EE007D8032E62D0122E60D0012E00D07CE04EE01A2E5AD039D80221182E72D074E01C010020D91F00009506002088040020E502002096
:402A00003001002000000A402120000000030020F40800000700C0FFD40800007F100000EC080000DC080000FFBFFF0348600000E4080000E8080000FFFF00FF78200000B9
:402A400090200000DC000A4064200000CC0800007804002008FCFFFF1F2E38D00321202E36D038E070236343019AD31842331B785BB2002B02DB20000CF0F0F90923002276
:402A80006343394939485918C318985C8D5C854221D30132092AF8D170236343344AD31842331B785BB2002B02DB20000CF0D6F9032E01D01A2E0ED10922100060432B4B33
:402AC0000021C0180CF01FFC05E0002100E00121200006F0CDFB2000FFF7FCFA0500002C40D11A2E30D004D8032E2DD0162E2FD038E0232E02D0282E1CD033E020000BF052
:402B00002DFF67300378012B2CD16B780F252B4228D02000FFF7DEFA43782B4202D183789B071FD00022134B1A731A7001325A705A6017E020000BF011FF67300378012B8F
:402B400010D16B781B070DD0002008F0DBF909E020000BF003FF67300378002B02D1AB789B07F1D10FB0F0BD300100209506002088040020C802002070231A00424370B5A4
:402B80000D00214904008A184B321278002A1DD0002D1BD1013520000BF0E0FE5C233F22FF33C35C9343C02B04D080212000C9040CF026F900221F212000FFF71FFD002D62
:402BC00020D00121200004F07FFF1BE0C82263439200CB1820001A86FFF7A8FA0121200004F072FF002DD6D080212000C9050CF007F9172120000022FFF700FD03492000FB
:402C000005F040F870BDC04688040020831D00001E39F8B504000800062900D9A9E00CF0BDF904A8227881A89E0020221F21200006F01EF9702363434E4A0121D318C82211
:402C400092005A86200004F03FFFF02363434A4AD318A8331B785B0700D48AE000212000FFF78AFF85E070252F0067431E21200006F05EF93F4E2000F7193B8E7B86483705
:402C8000FFF7DCFB3B782000002B02D104F0F6FD01E004F0A5FD654375194B352B78002B2AD020000BF05AFE9B3005780BF069FDB8235B006343314AD318314AFC335A66D2
:402CC000304B314A9A58D20714D509262F495A58B2435A505E58002D01D00822164301255A582A4332435A50294A2A499D505A582A435A500BF049FD2000FFF7F9F9437FF0
:402D0000002B33D001201F49234A8B5803438B502CE02000222106F00BF90121200004F0D3FE26E01D490A222000FFF7F3F8011E02D1200004F0C8FE1422C821524289005A
:402D40002000FFF7E7F8164B002802D10A22242101E001222221200006F00EF909E02000212106F0E5F82000FFF768FB2000FFF709F8F8BD880400200019000004030020DE
:402D8000C91D000000000A40F4080000302000003C20000044200000EC08000088130000112C000070B504000E000BF051F805005E2E0FD15D21200006F0BAF82000FFF7C3
:402DC0003DFB124B00219D4200D901212000FFF7D3FE19E05D2E17D10D4BC518FA23ADB25B009D4206D90B4B01223100200006F0C3F809E05E21200006F09AF82000FFF785
:402E00001DFB2000FFF7A2FB70BDC0468D12000072EDFFFFA52D000010B5040020221E2106F026F82000FEF7ADFF2000012104F04BFE80212000C9040BF0E2FF002220215B
:402E40002000FFF7DBFB10BD10B5040020221E2106F00EF82000FEF795FF2000012104F033FE80212000C9040BF0CAFF002218212000FFF7C3FB10BDF0B5D249D24A89B0E0
:402E8000D24B914201D8012200E00222D04C1A70200006F0CDF9CF4E002801D000F0DAFCCD4B9D6C2300B6331A782300B7331B781B02134301D100F0CDFCFFF719F90378E4
:402EC0003B2B01D800F0C6FCC44B9D4205D0C44BEB18012B01D900F0BDFC4378032B01D000F0B8FC2300AA331A782300AB331B781B02134301D100F0ADFC00210800FFF7DC
:402F000005F9C37833702300AC331A782300AD331B781B02134301D100F09CFC01210020FFF7F4F8C378B3702300AE331A782300AF331B781B02134301D100F08BFCE31857
:402F4000DB7873702300B0331A782300B1331B781B02134301D100F07DFC02210020FFF7D5F8C378F3702300B8331A782300B9331B781B02134301D100F06CFC0020FFF7A2
:402F8000A9F80378172B01D800F064FC01220025944B9A603F32DA603C3A1A613D32DA613C3A1A623D325A61403A5D629A624132DA622300B6331A782300B7331B781B02C8
:402FC0001343E318188B18235843013880B201F0CFFF854B85491A680F2309689A430909D2B20B401343824A113B13700C21FF220B006B430135F3189A751F2DF8D10021DE
:40300000082280207B4D7C4B29707C4E69701A607B4B073AB363F36C00061343F364F36A0343F3627264774B774A78481A60784B784A995019507848784958507849086896
:40304000039680B2029102990F68BFB2B842FAD00527734800689F5086B280219F5849020F42FAD00299096889B28E4202D980277F023943081A6B4908800020985062B623
:40308000694B6A491A688A4206D19868684E5A68921956425641801919600021654A59609860654B1A602300B6331A782300B7331B781B021343E3181A7D604B1A70E31CFE
:4030C000DA7F231DDB7F1B021343042B03D9043B9B10AB7000E0A970631CDA7FA31CDB7F1B0213430433E3186B60E31DDA7F23000833DB7F1B021343042B1FD9043B9B106B
:403100002B72631DDA7FA31DDB7F1B0213430433E318EB6023002A331A7823002B331B781B0213432B82230028331A78230029331B781B021343E3186B6102E000232B72CB
:403140002B822300C2331A783D4B3E493C331A703D4B3E4AFC335A638E22D20088583C4B002603408B502300DB34DA331A7823786E761B0213430F00B34212D007213000C6
:40318000FEF7C4FF417804004B1E99413000C9B20BF0F8FEA17830004B1E9941C9B20BF0F7FE2C4C002021000BF0F2FA0020FEF79FFF0530C27F284B022A4FD121004831A2
:4031C00019604DE0E0180000FF7F00006C0000200019000030010020FCF0FF0F012B0000FAD4FFFFFC000140E80F00F0EC0F00F07B060020B002002080E100E000000340C5
:403200006588EDAC4C000020D98C000018D00000001000E010D00000BF5D000014D000003C00034074060020000D0020EFBEADDEF4CFFC3FA98B0000700600208400002095
:403240008804002000000A40040300202DCC00001818FFFF50F30000F402002000221A6000248C4AC2218C4B002005F085FE039B20009C630BF0F2FAFA2251213435874B5C
:40328000520020002C7005F077FE642120000BF039FE834B4233029300200BF03DFB0222029B1B78134213D07E4A032100200BF0CDFB0F280CD00222029B1B789343029A60
:4032C00013701378802252421343029ADBB21370754C230035331B78012B09D100200BF03DFBA2300378072B02D100200BF06AFD00200BF033FB71300078C0B2002802D1AD
:4033000007F000FE7CE0637E063B022B6AD80020FEF7E0FE00250226644A07AB03901A800023320000931900180001F071FD002804D10C2204AB9B18585514E000230021F4
:40334000009332000533080001F062FD002805D10C21012304AA5218535504E00C2204AB9B180A3A5A550026012D01D00125D7E704AAE38C9589AB4207D1E38C49219BB253
:403380002385300005F0D4FD2CE0238D9D4211D0E38C474A9BB2934201D1012D07D8002328224921180005F0E7FD25851AE0E28C9A4217D04921002005F0A0FD002811D12F
:4033C000238D9BB2E384E38C9BB2002B03D180211800090104E0039B5B785B0702D5082107F0CCF930481C3001F0F4FC01000B2806D8637E2F4A9B00D3189B6A00209847DD
:403400002D4C2378002B0FD02C4B1B78052B0BD12321002005F072FD002805D1202105F06DFD002800D15FE21F4B34331B78002B00D1BFE00020FEF75BFE831DDC7F2233FB
:403440001B7834300593067800200AF02BFC039000200AF0EFFB2100049019480BF032FE049B184C184DAA2B32D9704364210BF09FFD3E592021F30ADB021843134B38511B
:403480002B60A823A922DB00F950D200BB580B43BB5032E0EE020000B1900000B11D00008804002001910000B00200200303000001020000D0F30000F8040020F00200206E
:4034C000C05D000074200000100A0020A14B0000059B642158430BF06BFDA8232021A9223E59DB00F60AF60230433851D200F950BB588B43BB5000232B600020FEF7F8FDD6
:40350000D94A05301268C37F0592002A20D0022B1ED100200BF022FA04000BF032F92300059072331B78002B0CD0D04B1B78052B08D1CF4B1B78002B04D19B342378002B59
:4035400000D196E20022CB4B05981A700BF01DF9C94B1B78002B00D058E3C84AC849BC5807221440062C1AD1C6480A58A243042422430A50C4480A58520405D4A823DB0065
:40358000CA580123520A93438022D2013A508021A8228900D200B950002B00D01EE30022BA4B512134331A70FA22B94B5200002005F0E2FC0023B54CA3630BF07DF9002817
:4035C00000D169E60BF0DDF8230034331B780390002B00D021E30222AE4B42331B78134200D01AE3E069002800D016E3472105F085FC002800D010E3482105F07FFC0028E1
:4036000000D00AE3492105F079FC002800D004E3627E072A06D1C02149007B580130FF3003437B508E21F020C9007B580003034388207B50984940047B5801260343922096
:403640007B50C000E11D3B58C97F1B0C02394D424D4133409D4200D0DFE2894B195823000833DB7F090A023B5D425D4131408D4200D0D2E2063AB24230D80223E58CFF3332
:40368000ADB29D421CD00ED8B54227D10023022219001800009501F0BBFB02230093002329001A0017E081235B009D420FD07B4B9D4213D1002300960222190018000BE003
:4036C0000023009602221900180001F0A1FB002331001A000096100001F09AFB704B1D78EDB2002D02D00125002693E00BF0FCF80028F8D028000BF031F972300378002B74
:4037000000D08CE25C4B1B78002B5ED10BF039F8594B04901D78002D54D14421614A0120BB5880260B43BB50C522D200BB583C318B43BB507832B9585B4B36060B40F0211E
:4037400009030B43BB503132FF32BB580343BB50BB588340C340BB50544A554B1A60E0229200BB588343BB50B958524B0B4052490B43BB50FA239B00F8507032BB5829000D
:403780000343BB502B00062205F02AFD4B20404203F0F2FC494A2800136833431360484ABB585B005B08BB500AF048FD454A2800BB581E43BE50444A444BB9580B40BB50F2
:4037C00001F070FD04980AF0E0FF2B4B1B78002B00D124E2032B00D121E26378002B08D03B4B1B6CA28F9BB2934202D0322002F0C0FF0AF0C6FF0421364B374A1B889BB200
:403800001360364A13680B43136030BF0AF0BDFF01252E0003980AF0B8FF002E01D00BF075F8002D00D137E5637E063B012B00D92FE50021080003F041FC0221002006F0C6
:403840008BFF0121002003F039FC0421002006F083FF1EE5224A234913680B43136002F0EDFFFFF793FBC046F4020020F0020020FA0200200005002000030020AC200000C0
:4038800000000A402C2000003C200000B0020020B11D0000880400209C04000001020000F8040020CC080000FFFF00FFDD5200007804002009F8FFFF43040000DC000A4003
:4038C00064200000F4080000D408000080EFFFFF0000034052F1FF0F0400034010ED00E0600000204C420000D04B20701B78002B00D199E5CE4B07AE1C880AF042FFCD4BBC
:403900000490FC330393039ACB4B04A9D366F02301225B00FB58A4B21343E032FF32BB500B235B18601D1900320003F02FFAD620C0003A58C14B1F241A403378C04D1B046A
:403940001343E822D200B958BE4A0A4004A9C97A214089020A43E821C9007A503B50F023F0220121DB00FB58D2005B005B08BB50B54A0A20BB58FC245B005B080B43BB50DF
:4039800002F0F7FEE4229200BB58B0499B0A9B02BB50BB58A4000B43BB50FA2310229B00FA503B5913433B5104980AF0EEFEF8239B00FB589E4B1B88192B00D834E59C4B42
:4039C0001B889BB204930AF0DCFE039AA04B05909366F02302225B00EB5804A91343DF32FF32AB50049B3200581F0B235B18190003F0CCF9D822FF21D200AB588B43317821
:403A00001F261943E823DB00E858924B184004ABDB7A33401B050343E820C0002B50F023A9500121DB00EB58C0325B005B08AB503032AB580A205B005B080B43AB50E522D6
:403A40009200AB5884499B0A9B02AB50AB580B43AB5002F08EFEFA2320229B00EA502B5913432B5105980AF090FEF8239B00EB58DAE47A4B1878002800D063E50AF06EFF7B
:403A80009B3004780126002C28D1754A754B15681B8E2A889A4209D26A8834009A4205D20021AA8802349A424941641A0A260398E98870430BF006FBC0B2031C092800D999
:403AC0000923049ADBB26643AA2A04D9AE19F51834352E7802E0AD19ED182E7B604B1A68137AB34266D260490B68002B0BD18024A823A920E401DB00FC50C0003B582343D5
:403B00003B505A4B0B60D588039BAD085D19584BADB2DB8EAB424DD90AF033FEFC240122E40004903B5904A9934380223B513B59120613433B510B235B181900280007AAFA
:403B400003F024F9D620E8251F21C0003A58494BED001A4004AB1B7B1B021343039304AB7A59DB7A8A431940114301227951039B3B503B590A2013433B513B599340D340F6
:403B80003B5102F0F6FDE32225219200BB589B0A9B020B43BB50354A374B1D391A60FA23FC229B00F9509200BB580B43BB5004980AF0EBFD314BFB585B019B0E01339A1BE0
:403BC000D2B29E4201D9F31ADAB2002A00D1B9E400223100100001F09BFCB3E40AF0D1FD0121274C05003E593B59154A0B4205D0135932208B43135102F0BBFD002001F01B
:403C000071FB3E5128000AF0C0FDC8E401211D4A13784B4000211170BEE40025F9E50AF0B0FD0421184A13688B43EDE57C0400207E040020040300200D540000FFFF00FF08
:403C400000000A40FF83FFFFE4070000E5030000C9530000FFFF0FFEEB03000000050020F402002088040020FC0400208D540000B0020020FF00FFFF140A0020B0200000CD
:403C8000EC0800000103002010ED00E0F8B59324A4004443164D02272C19164D6619002535708326B600A6193770134EA6193170124961180D80124961180D70852189009C
:403CC00061180B6084239B00E3181A8086239B00E3181D7087239B00E3181D6088239B00E41801235B422380182107F04BFDF8BDB00600200B0200000D02000012020000A7
:403D00000E02000070B59324A4004443164D2C19164D6619002535708326B600A6193570134EA61931701B26124961180E80124961180D708521890061180D60842189005D
:403D400061180D808621890061180A7087229200A218136088239B00E41801235B422380182107F00FFD70BDB00600200B0200000D020000120200000E02000070B59324B1
:403D80000500A4006C4308F02DFC0E4E2800A259042107F0BDFA00210B4A33199A1811708E2292009B1803221A708E239B00E218921928000F310BF077F82800172107F085
:403DC000E1FC70BDB00600200702000070B504000E000AF0ADFE0500062E09D0082E23D0022E24D164220921200007F0C3FA1EE04021200007F068FB002815D02B00703366
:403E0000197850331B6820009B69984700237D352B7093239B006343054A20009B5803229A70FFF7ABFF02E0200007F008FD70BDB006002070B50D0004000AF079FE022D79
:403E40002AD1030066331B78144D012B0CD1020081321370932300229B0063431049EB1880305B1802701A70200007F0BFF993238E219B0063438900EA18521803211170D3
:403E80008E2292009A180B312000AA180BF00CF81721200007F076FC70BDC046B006002002020000F8B50E0004000AF041FE93239B006343404A4149D31807005B18B01EED
:403EC0001D781600062876D80BF068F8040A1416187563002A000021200008F03DFB6AE02000032102F040FC1B220921200007F041FA60E0002157E0012143E008212000E2
:403F000007F0E2FA00280BD093239B0063432000F258042107F0FCF9200005F013FE4AE02749200007F0D0FA011E2BD00B2D16D193239B006343F35804359B78102B12D1B3
:403F40003B007033197850331B6820005B69984701237D373B70200008F044FB03E00A3D6B1E9D410D359327BF0067432000F259042107F0CDF9F2592900023220000AF02A
:403F800093FF14E0200002F0EFFB200007F01EFC11E0132D03D1200007F08EFC0BE0102120000AF073FF0221200002F0DDFB1721200007F0E7FBF8BDB006002047020000EE
:403FC0001010010093239B004343174A10B5D318164A9C18002222708324A4001C192270134C1C192170134959180A80124959180A708521890059180A6084218900591873
:404000000A808621890059180A708721890059180A60882292009B18012252421A80182107F0B0FB10BDC046B00600200B0200000D020000120200000E020000F7B504001B
:404040000AF076FD93239B006343274A01909E581500B7780F2F35D801210800B840234F384240D11827384226D1163F40062AD5D3181F4A9B1819701E498B7C002B04D1EE
:4040800010212000FFF79EFF2DE0F388DB05DB0D022B0AD1B368DBB2002B06D14B7C087C1B0203438A7C5B1801E01222124B07212000FFF7EBFD16E0D3180D4A0F009B1861
:4040C000197000E0022701981B229C3007700921200007F04FF993239B0063431E21EA5820000AF0E1FEF7BDB0060020A6F000000A020000001900007000002010B504007D
:404100000AF016FD943003780421012B00D90C312000FFF757FF10BDF8B50D0004000AF007FD02000300C032A81E126806284BD80AF034FF040F1616164A1A007033197835
:404140002000536998470A220921200007F012F93AE001227D331A702000FFF70FFE33E0200007F06CFB2FE0D36920009847011E23D093250026AD006543062200212000E9
:4041800008F0EAF9114B20005D19114BEB181E70104BEB181E700AF0CBFC070037220321200004F07FFF3B00012281331A700A4B8037ED183E702E7006E0200002F0D4FAC3
:4041C0001721200007F0DEFAF8BDC046B0060020070200000902000002020000F0B585B004000AF0A5FC00210390200002F0BCFA0921200004F09CFE80219327490020005E
:404200000AF096FE17220021BF00039B6743A233AE4D1A70AE4AEB199B181970200007F053F92E00011E00D1A3E020000AF080FCBB5905009B78981E142800D93BE10BF055
:4042400075F87D0020012A012A01200115007D0024002400240020013A013A013A012A0130004A007D0086003A017D0093239B006343F618964B6735F61801232A780B210A
:4042800033709A4200D016E107E09322142192006243B6188F4AB6183370200007F072FAF9E093239B006343F618894B0221F618012333708223AA7AFF337F2A02D9EA5CA6
:4042C0000A4301E0EA5C8A43EA542B006D33FF33182201212EE093239B006343F6187C4B2900F618012385313370FF31200002F0EFF96821FF316A5C102013002A0083437C
:404300006B549B321278002A01D003436B546A21FF316A5C022013008A2283436B54FF32AA5C002A01D003436B542B00062202216533FF332000FFF7A9FCACE093239B0071
:404340006343F618624BF61801233370B3E093239B006343F6185E4B8535F6180123FF3533702900200002F0B3F92B0004220C21E0E77E59584B012200930300300007F07D
:4043800001F8002800D180E020000AF0D1FB03007F590600B878673301381B780E2800D989E00AF0FBFD6E080F6E6A8888888888888888882F00012B7DD17B780D21012BC9
:4043C00079D16AE7320075321278012A63D13200733212789A425ED132005132FF32002B00D0043A7023D2781340102B53D10F22FB7A05219343802B00D14EE70621502B51
:4044000049D14AE73A78002A45D1932583210420AD0065432D4B89005B19591808702F49023059180A802E49113559180870284920005B1880211A7009010AF079FD234BAA
:40444000FF35ED182422390028000AF053FF3300C0331B68234ADB6B29002000984714220921200006F086FF8021200049000AF05FFD1823A23633700DE094363378012BED
:4044800019D9200007F0A2F905E03378002B02D17379DB0913D1039BA2331B78172B12D10921200004F02AFD00280CD1042120000AF032FD07E02000FFF720FEEBE7200006
:4044C000FFF7BCFDE7E705B0F0BDC046B00600200A02000047020000FFFF0000120200000B0200009DB10000F0B585B00D0004000AF01EFB0600A81E072800D9BDE20AF0D4
:4045000015FF0800BC02BC02BC024000BC0226007B00330094331B78012B00D8ADE2330067331B78012B00D0A7E233008B331B78012B00D0A1E2AC33FF33F35C002B00D023
:404540009BE205220921200006F014FF95E233009C331A78002A03D0002204211A707EE03300A4331B689B0500D586E2D6235B00F35C002B00D080E20221200001F066FA0F
:404580007BE235009C352B78012B06D10921200004F0B4FC002800D0F4E00021200029700A0006F0B5FE330094331B78012B16D9330067331B78012B11D133008B331B7811
:4045C000012B0CD10B21200004F0B2FCD6235B00F35C002B03D10221200001F037FA2000092104F0A5FCC021200089000AF0A0FC2000FFF7F3FD40E220000AF099FA0300E6
:4046000084331B780700019303009C3303931B78060009212000CC3702933D6804F088FC8021200049000AF083FC330094331B78012B1FD9019B052B1CD0029B002B1CD1F4
:404640008B363378012B0ED00121200001F0FEF912220B21200004F025FD8021890020000AF05AFC09E20B21200004F047FC002811D0F2E7029B002B0DD093239B0063437E
:40468000D84AD318D84A9B186A46127A1A700023039A137008E093239B006343D14AD318D14A9B1800221A70019B162B00D9E4E118000AF03BFE1700E20158002300E20192
:4046C000630067006B009600CC00D500DA00E500320130004C001301A901DE01E201E201E2013F0020000B2107F04CF82000032102F03AF8200006F0D7FDBEE193239B0092
:404700006343B84A0821D318B84A9B1802221A701023013A0AE093239B006343B14A1121D318B24A9B1802221A7013002000FFF7E9FAA2E193239B006343AA4A1621D318FA
:40474000AA4A9B1802221A7080231B02EEE793239B006343A34A1221D318A44A9B1802221A700423E2E793239B0063439D4A0E21D3189F4A9B1801221A7076E1200007F05F
:404780005EF87AE1200007F021F876E193239B006343944A0320D318964A991800220A708321890059180870934959180A70934959180A80924959180A7085218900591897
:4047C0000A608421890059180A808621890059180A708721890059180A60882189005B1841E12978200007F0EBFE93239B0063437C4A2978D3187F4A0D209A181170832280
:404800009200991800220A707B49591808707B490E30591808807A4959180A708521890059180A608421890059180A808621890059180A708722082192009A1811608822C4
:4048400092009B18012252421A8010310DE193239B006343634AD3186A4A9B1809220CE00121200001F080FF07E193239B0063435C4AD318634A9B180B221A701521F4E023
:4048800093239B006343574A2978D318594A28799A182E7B117083229200991801220F270A705549103559180F70544959180E805349591808708521890059180D60842153
:4048C00000208900591808808621890059180A708722802192009A18090281E093239B006343404A2879D318424A0126991800220A708321890059180E703F4904365918A5
:404900000E703E49103559180A803D49591808708521890059180D6094E03B6858780338082829D893232F499B000AF037FB091025192505052121008021022289001DE05B
:4049400063432A4ACB189B1802221A7006E06343264ACB189B1802221A70013A20210DE06343224ACB189B18022280211A7005E080210222090101E0022200216B886E7886
:404980000193AB6817480293932384469B0063431848634484469C4460462F782D7B0770832080001F180220387013481F1813483E701E183580002611481D1806302E704C
:4049C0001D180298286084206D468000AD88181805808620800018180270872292009A1811603BE0B00600204B0200000A020000060200000B0200000D02000012020000F7
:404A00000E0200004702000093239B0063431C4A3968D3181B4A0626981800220270832080001D1801202870174D10315D192E70164D5D192A80164D5D192870852080007C
:404A4000181801608421890059180A808621890059180A708721890059180A60882292009B180122524218211A80200006F08AFE03E010212000FFF7A5FA05B0F0BDC0460D
:404A8000B00600200B0200000D020000120200000E020000020010B50749084C084B6058013A034012051A4362508022635812031343635010BDC0469020000000000A407E
:404AC000FFFF0FFCF8B5060009F048FF723003782D4C002B02D10C21002336E02378052BF9D12A4A2A4B2B49D35815005B019B0E0133012B32D160685D30007800282DD034
:404B000080255058ED0528435050257A627A954229D29A4200D96372637AAB422BD3637A9D42D8D029D2013B6372677A3800FFF7B1FFBD4223D0636836215C331A783000F8
:404B4000154B04F019FA0C210123A372002B19D1E368002B16D03000984713E068580F4A02406A50D1E7934205DB9A4200D26372637AAB42D3D96572D1E70133D4E70021DB
:404B80000B00E2E7F8BDC046F002002000000A40B0200000A8200000C54A0000FFFFFFBF70B50500FDF7A4FA0400280009F042F8A92808D804480549283443582278DB0ACB
:404BC000DB021343435070BD00000A4074200000F0B583B00F000192134A166802231E43126815009D43002306220021012004F0F7FA002F15D00024019B043B9BB2019334
:404C0000094B1E60C046C046C046C046C046C046C0461D60019801F0ACFD0134E4B2A742EED103B0F0BDC0460000044070B5050009F00EF9124A134B904201D801221A746B
:404C40001C7C012C05D0104A08240621904201D804E008210D4A904208D800E00C21012228005A742732FFF7B3FF01E002221A742800A2B2064B372104F07EF970BDC046AF
:404C8000AB0D0000F0020020A60E00009F0F00002D4C000010B50400032103F035FE032120000AF0F3F810BDF0B585B004000E0009F03EFF03000190C03320001F6802F004
:404CC0007FFA03AD2880012E02D0052E0BD024E000212000BB6998472000BB6931009847322001F046FD200002F06AFA019B2880703319786A5C002A09D1019B200071339A
:404D00001A7002F0B9FA2000FFF7C4FF05E0044B01221021200004F02FF905B0F0BDC046495900000023F0B585B00D000600039309F027FDD022244CD200A3588021019376
:404D4000A0230905DB00E150B8235B0073431F496D04CB182933FF331978C023DB0207002B40002901D01A4D01E08025AD002B43A350E02201215200A3580B43A350802115
:404D8000A0220905D200A3580B4206D1039BC72B03D8039B01330393F5E7022001F0E9FCE0235B00E5588022A0231205DB00E2500199300001F000FF380009F0E6FC2D0C61
:404DC000E8B205B0F0BDC04600000A40F00200200002080070B50400202509F0D2FC002C12D02368002B0FD000230126216832009A40DDB2114203D023689343236003E018
:404E00000133202BF3D11D0009F0BFFC280070BDF0B501258DB007922A008A40089312AB1B780400019343009A400E00059209F0A8FC4A4F0B902300002E17D1C133FF33FF
:404E40009B00DA190692FB58019A0093AA4205D041230493313B0293039505E049230493393B0293019B0393EF2615E0C533FF333A4A9B009A180692FB58019A0093822350
:404E8000012A00D19223DB01049380235B010293EF26092336020393304BA400E4188E238022DB00E3582E4909937B5892010A93089B00985B041343079A0791D20313433D
:404EC000284A02401343089A002A02D08022520301E0D82252041343069A0A20136001F048FC214B019AFD58059B1D406B1E9D418E23EDB2DB00002A0FD1069A00990A20C2
:404F00001160E258B243E250099AE25001F031FC124B079A0A99995016E00299E2580E43B243E2500398019AE15882400A43E250E25804990A43E250079A084B07999B5852
:404F4000059A1343054A5350084B059AFA500B9809F01BFC28000DB0F0BDC04600000A409C040000FF1F10FE8C040000940400000723034A000211680B40184310607047C6
:404F80000C03014070B5B8240600640074430F48041923002933FF331B780500002B0CD002213000FFF7BEFE011E06D09620C00209F0FEFFFE3480B2A085B82040007043FF
:404FC0002818FE30808D80B270BDC046F0020020012170B5104A114C9025A35832208B43A35080239B01E25849180A43E250E2582D018A43E2500022E25001F0BAFB08221A
:40500000635932209343635101F0B3FB032263599343635170BDC046EC08000000000A40802330B5114A124C9B01D358100015590B290FD801228A400E490A4206D111053F
:4050400006D4520506D50C4A134003E0954301E05B005B08002D04D1084A134201D101229343802292018350055130BD00000A40042000003F030000FFFFFFDFC000F8FF1F
:40508000F023434370B5184A0400D318A8331B785B0728D509F075FB144D06002B79022B03D100212000FFF7BBFFFA22012180240F4BD20098582406884398509858204380
:4050C0009850E02080001C580A4A22401A5070301A588A431A50FA229200995000233000AB6009F052FB70BD001900007004002000000A4008FCFFFFF7B53D4C1F0008AB03
:405100001D7823790E000192022B02D10021FFF787FF384B0198A36070432771642109F0D1FF354B80B2354E984203D9344B98420BD800E03348052109F03AFFC5228021E6
:40514000D200B35880B20B4308E00A2109F030FFC5228021D200B35880B28B43D427B350FF00F259284B0A211A40C838019209F0A9FF019BFA2200041843F0510127D2006C
:40518000B3580A203B43B350B358BB40FB40B35001F0EFFAE0239B00F258BA43F250F2581A4B1340002D06D0194A013D13436D012B3A154000E018251D43E0230121FC2012
:4051C0009B00F5506833F150800033580B4A0B4333502379022B0AD18024A40110590D4D0D4B034050590B43014351511351F7BD70040020792B00001B0C000000000A40D9
:40520000282300001C0C0000FFFF00FF09F8FFFF0B04000004200000FFFFFDFF002382B00330009301930090009B032B06D9009B043B0093019B01330193F5E7019802B0F3
:4052400070470000A022F0B5144B52009A5C4020D2B214009F25124E0834FF306D00A24213DA1F5C595D8F4216D21700195C1837BF000231BF59890059188F61195C013243
:405280000131C9B21954D2B2E9E7A02149005A5C50424241D2005A54F0BDC046F002002000000A40E021012210B50A4B89005C5894435C505C5814435C50FC2468315A5004
:4052C000A400195911431951034B37211A74FFF7ADFC10BD00000A40F002002010B5FFF7E1FF10BDF8B509F04CFA07000C4C266802231E4325689D4300230622002101201D
:4053000003F06EFF2660C0462560002306220A21012003F065FF380009F037FAF8BDC04600000440F7B5274C050023181B7B0191002B45D001F0E4FC280001F005FD2800D2
:4053400008F0B0FC052109F033FE052358436E00A319DA8980B2DB89904201D9C31A00E01B1A9BB2322B01D9A319D881A719FB89142B0DD9F88983B228000093FCF7B8FE99
:40538000009B008A6421584309F012FE388203E01423FB8100233B820A21019809F008FEA3191A8A80B2824200D91882AB00E3185B69002B04D0A419E189280089B2984711
:4053C000F7BDC0467004002070B50E4D04002B181B7B002B14D070232A0043431832D318198EFFF79FFF2000FCF7A0FE6300ED18EB89053B9BB2EB81034B1C19012323727E
:4054000070BDC04670040020F004002070B50E4D04002B181B7B002B14D070232A0043431832D318198EFFF77DFF2000FCF77EFE6300ED18EB8905339BB2EB81034B1C19B5
:405440000123237270BDC04670040020F004002070B50C4D04002E18337B002B10D001F04FFC200001F070FC00236200AA18D3811382A200AD18044A337314196B61237245
:4054800070BDC04670040020F0040020F8B5040009F077F9194F0600BB7A002B07D0FD68002D04D13621200003F042FDBD72144D144B7A68EB58107A5B019B0E0133984291
:4054C00001D2FFF7E7FA104BA4001C191900E368002B0CD08022A823D201DB00EA50A922D200A858094B0340AB500023E360012330000B7409F049F9F8BDC046F00200209E
:4055000000000A40B0200000F0040020FFBFFFFFF0B585B00E000292050009F01FFA00902800FCF7E5FD0530C37F0027019309F028F9184C039036212800A77203F0F8FC9F
:40554000029BE360019B022B01D00C241CE0009B72331B78002BF8D02378052BF5D10E4B0E4AD35826725B019B0E013363729E42EBD00123A372636836215C331A7828006D
:40558000074B03F0F9FC3C00039809F0FEF8200005B0F0BDF0020020B020000000000A40C54A0000F7B50400019109F0C1FA030005000198C0331E680138593B1F7805288D
:4055C00000D91CE109F0B2FE0600BB001B01680058002F002B0073331F702321200009F055FC2B0001227D331A700D3B1978C023834ADB00D058002901D1824900E08249CD
:405600000140D15009F0BEF9002808D009F0BAF97E4B02000F21200003F0AEFCEFE00F21200003F085FC012F00D0E8E02B0078331B78012B05D12B007033197820007369D3
:405640009847012720007368714972359847200002212F7009F01AFC2000F3686D4998476A4B2000FA22102103F086FC09235C43694B1133E754C2E009226243664B1133EB
:40568000D35C012B18D1AB7C0321012B00D10121200003F039F9B2E01021200003F048FC2021200009F05CFC09235B4D63432A0011329F5C012F03D02000FFF7EBFA9EE0CD
:4056C000200009F035FA1422C030036852421B6A4F49200098470028D9D0336A14224C49200098470028D2D1200009F021FA837B012B21D1C0236F300178414ADB00042049
:40570000002902D1D158814301E0D1580143D150200009F00DFA0600200005F039FF33000722A2331A700423A4363360002C66D16035FF352C7062E0773007705FE0F3698C
:405740002000984700210190B3692000984701212000B36998472B0000270122B4331F604A3B1F7020001A711F7205F09FFF2B4A1521200003F096FC09236343264A10219F
:4057800011329F54200003F0D3FB1621200003F0CFFB7021200009F0E3FB2B781E4F012B1DD1019B002B1AD0C2227035287814251349D2008B582B438B50103A8B5800284A
:4057C00002D1A020C00301E0A02000040343144803408B502000042103F096F805E00B4B01221021200003F0C7FB092363431137FF1801230B493B72200033699847F7BD1F
:4058000000000A40FFFFFFFEFFFFFFFD49590000881300003F590000F0040020D5020000FFFFFFBF2D5800007047000009235843024B1818002303727047C04601050020B2
:4058400010B5040009F074F9030072331B78002B0BD0030067331B78012B06D19621C030036849009B682000984710BDF8B506000F0009F05DF9020086321378012B0AD1FE
:405880000025C830036804001570AB4203D03900300098472560F8BD70B505000E0003292AD109F045F9030080228E331B880400520093423DD005D8002B0ED00022012B8A
:4058C00039D034E00222FF3293420ED0013293422DD1023A0023FF3A2DE0280009F04CFB002824D1042605210CE0280009F044FB0621002806D01AE001291FD1212109F043
:40590000C5FA1BE000231A0020006F300270012042402000703002702200743213711670280002F0F1FF00236E34237006E0002300E001231A0001260721E5E770BD10B502
:40594000102109F001FB10BD10B50400102909D1103109F0F9FA09206043054B18180023037104E00F2902D1313109F0EDFA10BD0105002010B5040009F0DAF80200094B3A
:40598000923213802B3A1278002A00D0064B020090308E321380112103801422200003F067FA10BD0404000002020000F8B5050017000C0009F0BCF8030006008B331F7031
:4059C0003A002800210001F073FC21002800341901F052FC220002238E32903413702370F8BD0000F8B506000F00012929D109F09FF809237343134A0024D318020005008E
:405A00005C709A325C71104B14702100220030009F55FFF7CBFF220039003000FFF7C6FFC82000F0A6FE2B0067331F70013B1F703000FFF79FFF2B0072356E331C70DC700B
:405A40002C70F8BD01050020EC0B002070B504000D0009F06DF8030067331E78012E16D124331D701A3B1978C9B2002906D12A00200001F01DFC2A00310002E02A006F301C
:405A80000178200001F014FC322000F072FE70BDF8B5002009F04CF8030087331B78002B32D0B0217C22194C8900635893436350AE239B00E250030071331D78EDB2002D9F
:405AC00022D10A3B1E78012E0BD18B30070002782900280001F0ECFB3A783100280001F0E7FBA9200A4A0B4BA15880000B40A3502258094B09491A400A432250AA229200C9
:405B0000A05803400B43A350F8BDC04600000A4004060000FFFBFFFFFEFBFFFF10400000F7B5070009F004F8030087331B78002B00D1A8E00300010071331B78524C6731AE
:405B4000012B27D1AE251026B022AD0066519200A3583343AA26A3500978B600A359012900D090E074300078042800D188E007218B4303390B431C31A3516151A3580B4322
:405B8000A350AD239B00E3585B057CD5AF229200A35872E0C026F600A2593C4B134010221343A3510D780021012D69D1A259384B8B301340A351037836499B005B5CA259E9
:405BC00059025B010B431343A3510A2000F0D1FDAD2380219B00E3582F4A0193A358C9000B43A350A2592D4B80201340A351A023019A5B011A4040010226824208D0019A07
:405C000013408B4202D12E00013501E0022635000A2000F0AEFDA92189006258204B680013406350F302625818431E4B134303436350AE237C229B00E250B0220C21920095
:405C4000A3580B43A350AD239B00E3580193019A1023022D02D11A4202D00AE01A4208D04023019A022E02D11A420CD001E01A4209D1AF2204219200A3580B43A35002E09C
:405C8000380008F091FAF7BD00000A40EFFEFFFF1FF1FFFF1CF4000004060000FFFFFFFCE8A3FFFF0104000070B50D00040008F03FFF012D17D1030072331D7074305D7168
:405CC0000378042B05D108F057FE01002000FFF7BDFE2000022109F0D9F814221521200003F0E0F90FE0022D0DD10200002372327730137003210370200009F0C7F803211E
:405D0000200002F001FE70BDF0B5160087B005AF3980050008F00CFF092334006B432C4A113CE4B2D3181B19029300230100029A8E319371274B3F5D1A68274B04911A422D
:405D400042D1A023254ADB00D3589B053CD40419230022008E3303931B7890320192BB4209D1019A31001370280003F0E1F80123029A937128E0019B1B78BB421AD0030088
:405D8000713319788C2201290DD1010074310978032908D81B78813A012B04D167300378012B00D1093A31002800903403F07AF9277009E03100280003F0A0F8002803D141
:405DC000019B039A1B781370049B188807B0F0BD01050020A4000A400720000000000A40F0B58BB0040008F0A3FE0490200008F09FFE03006E331B780500DBB20293030005
:405E00007A331E78F6B2002E00D0A2E046331F683D3B1B78059303006F331B782000069301F0CEF96B4618802B0082B28C331A8001230793059B032B0BD081B211222000BD
:405E4000FFF762FF6B46122219882000FFF75CFF07966B461978009B1B041B0E012907D01E00012B0CD06A4600261288B24207D10126994204D1200009F07EF84640F6B21B
:405E80002B008E331B8809AA13802B00713303931B78002B3FD1029B002B5AD1079B002B24D0002E55D0059B032B14D1200008F03FFE029982782000FFF778FD200008F093
:405EC00037FE012182782000FFF770FD0A221521200003F0E7F82000022102F015FD00236E352B702000FFF745FD32E01388D9B21A0A012905D0012A00D1BDE0002B00D08B
:405F000096E0914200D0B7E0200009F035F8002800D1B1E08CE0029B002B1AD1069BD35C022B0BD074352978042912D1002B05D1069B59424B41D35C002B0AD00F21200043
:405F400002F0F6FF00230421039A1370200008F0FBFF0498A830FEF73DFF0100072800D9DDE054D1200008F0E3FD050008F009FC2B008A331B780600042B44D8180009F059
:405F80000DF8030303383E00664AD3182A001B7C8332AB701278032A26D02A0075321278002A21D12A0072321278002A18D02A0067321278012A13D12A008B3212789A42FA
:405FC00006D9594B8C221621200002F0D5FF07E02B009621C0331B6849009B6820009847A9782000FFF732FD01212000FFF73EFC09E0092363434D4AD31801229A70012165
:40600000200008F0A1FF300008F0BFFB87E0002804D10131200002F077FC80E0049B414A83331B7820009B00D3185B69984776E0002E8ED11521200002F060FF002804D009
:406040006A463B4B12889A4283D1200008F070FD83300378022B04D10321200002F054FC05E01021200002F049FF0028F4D02221200008F00BFF6CE71521200002F058FF32
:4060800009AB1A882B0090331B889A4200D060E7C82100223B6A8900200098470923234A6343002816D1D3185871BB6A200098471421200002F03CFF0123039A13702B00B7
:4060C000A1331B78002B03D0072383352B7040E708213BE7D5186B78002B00D039E76B79002B0AD101336B7120007B6A984732221421200002F0D6FF2BE71421200002F0BA
:40610000FDFE061E00D024E7BB6A6871200098473100200008F0BAFE01236B7019E70BB0F0BDC0461CF4000041580000010500200202000070B5050008F0FAFC0300A83331
:406140001B680400002B01D001201FE003001521833328001E7802F0D1FE0028F4D1731E012BF1D9053E022E10D812221021280002F0A4FE0028E7D109236B436F34044875
:406180002278C018801883790120584070BDC04601050020F8B504000E0008F0C9FC03000500C03320001F6805F080FA002C1BD1C022C021204BD2009A58204BC9001340A9
:4061C0001D4A20005350210001F056F8C022C021194BD2009A581A4BC9001340164A20005350012101F048F8164A134B20009958154B0B4010498B50BB690021984701213F
:406200002000BB699847002E14D13B6931002000984718220F21200002F02AFE2B0083331E7025331E60363B1E70013B1E7001236E352B70F8BDC04600000A40FFFFFFFE40
:40624000FFFFFFFD04060000FFFBFFFFC02110B504008020094BC9005A580006024314205A5010315A5802435A5020000021FFF791FF00212000FFF7F9FA10BD00000A40F6
:40628000F8B5070008F054FCC1220821C026384CD200A358F6008B43A350A35952185B005B08A351A3580C318B430500A350322000F05FFA0A228021A359090213432D4A96
:4062C000A351A35801260B430221A3502A4A1820A3580B43A350C43AA35805318B4333432649A3506358334363504D39FF396358B340F340635063580343D6206350203136
:406300006358C0051B021B0A03436350A1581C4B32200B40802109010B43A35000F029FAA92080002258174B17491A400A432250AA229200A05803400B43C021A350083A0B
:40634000A35889030B43A3502B006E331E70053B1E70380005F0AAF92B00032283331A700223A8352B6038001B2108F08FFDF8BD00000A400406000094070000DC070000C1
:40638000FFF1FFFFFEFBFFFF10400000F8B504000E0008F0CDFB0500012E22D103000F21C03320001F6802F0C3FD092363432E4AD3189B78002B06D12A00723213703100B7
:4063C000200008F063FD01216E3529702000FFF7E1FE3B69254920009847254B254A102133E0331F012B34D800212000FFF7D2FE092363431C4AD3189A78012A1FD100229B
:406400009A702B00A1331B7893420CD1C0218020194BC9005A580006024314205A5010315A5802435A5001212000FFF71FFA1A21200008F02BFD002387352B7012E0012347
:4064400032220F2183352B70094B200002F094FD08E0062E06D120000121FFF707FA2000FFF70EFFF8BDC046010500203F590000495900007102000000000A4010B5024B15
:406480008200D358984710BD6806002070B51D2900D089E0454B1979012942D15A79102A13D0002A01D1597101E052005A715A79102A01D910225A71F22103253C4CC900CE
:4064C00062585A7992002A4362509A79102A19D0002A01D1013200E052009A719A79102A01D910229A717E21314C324D62598A4311009A7992000A432F49625162585200FB
:40650000520862505A79102A05D02C4B01221D2102F032FD48E09A79102AF6D100221A7142E0D97901293FD15A79012A0FD0520801D05A7100E05971F2247C211C4DE40060
:406540002A598A4311005A7992000A432A519A79012A0DD0520800D101227C21144D154C9A712A598A4311009A7992000A432A515A79012AC9D19A79012AC6D1F221032544
:4065800002240B4AC90050580B4EA843204350508020915900060843905106481158A943214311500022DA7170BDC0466806002000000A4094070000DC0700008D6400009D
:4065C00070B5050008F0B4FA0400280008F0F8FB2300943318705870987093200123800068437C342370044B181892239B00C0180023037070BDC046B006002093239B0096
:406600004343204930B55A1804325A50AC22520042431D4901258B181C005634FF3425701D00002457355833FF35FF332C701C70A04225D1154B5350154A164B16491A6098
:40664000164A174B1060174A5A60174A11600F21164A1160164A1E31FF3111601549164A1160A121C9005858144A02405A50144A144913689BB20B431360134A134B1A607D
:4066800030BDC046B00600200C05002095B1000039890000040300200F020000A8000A4000000A40000FF103B4000A40BC000A40D0000A400A404101D4000A40000408C0CD
:4066C000E8000A4002000F7E41004100C0000A40F8B505000E0008F02BFAC0300400036828005B6C9847236828001B6C9847142100B208F0E7FC93239B006B43154A04B254
:40670000D318154AE7B29B181A783F2324129A43E4B20023C02A0DD10121104B104A9A580A420FD00F4A9B589B070BD5280008F073FB0823002E0BD0FF2237707470B270E9
:40674000F37005E00021280008F066FB0023F1E7F8BDC046B00600203702000000000A40F40800003820000010B5002204F0D0FD10BD182310B5584307F0FAFF10BD0000FF
:40678000F8B517000C0008F0D3F9030067331B78274A012B36D00021012C01D1882149003C000025D219537B127B5B02520113430B43C022FF211F4ED200B05809010140D1
:4067C0008B4209D0B0581C490140B150B15832200B43B350FFF7CDFFAD239B00F3585A0503D50237002D06D01FE0DB0405D50124002D1AD13F19FCB217E06B425D416D42C1
:406800002C4012E0012C0ED1882464008B30017801258900535C521852785B015202134323430224C5E70024F0E72000F8BDC0461CF4000000000A400FF0FFFF034A044913
:4068400013689BB20B4313607047C0460CED00E00400FA0510B508F021FD03680C2B00D1FEE7064B9B68002B02D0012100209847034A044B5A60FFF7E1FFFEE768060020B2
:406880000C3003C0000D0020F0B585B0029072B6FEF79EFB7C220025304C314EA3599343783A1343A351029807F0D2FA2D4B984250D907F066FF80212B4A03901368090697
:4068C0000B431360294AA3585B005B08A350029807F0B4FC002306221900012002F080FC8F2280211201A35809050B43A350032301936420FFF73DFF38221D4F6420BB68F8
:406900009343BB60FFF735FF3822BB689343083A1343BB60019B013BDBB20193002BE8D1039807F032FF134B9D4208D8632D04D90122A3599343A35106E0002D04D1032216
:406940000025A3591343A35101350B48ADB207F00FFFA8E7FFF772FF05B0F0BD00000A40940700008C0A0000DC000A406420000000000440E7030000C05D000010B572B60A
:40698000FEF726FB0449054A8B585B005B088B50FFF754FF10BDC04600000A406420000010B507F0EEFE0121034A13688B43136007F0EBFE10BDC04600000940002370B5A8
:4069C0003E483F4C3F4D9A002100032B00D8A95801338150172BF6D172B6002408223A4B3A4D1C603A4B1A60C3223A4B12011A6012232B6007F0C5FE0722374906000B689A
:406A000093430B60354B36491B78DBB20B6035490B6893430B603449344B0A6818787F239A43034013430B60322007F0A1FE300007F0ABFEBC212E4A2E4B89011A602E4BD5
:406A40002E4A2F481A602F4A11602F4A2F491A609C2292010A602E4919602E490A602E4A2E491A60B82252010A602D4919602D490A602D4919608021490001602B481860D8
:406A80002B4801602B4919602B490C602B4919602B490A602B4A1A6003222B4B1C602B4B1A6011232B602A4B1A68A24200D11A600121284A13680B43136070BD0000002072
:406AC000556800000018000000000240300010400000044008000440080F0340E5F1FF0F0C0F0340100F0340180F0340CCF1FF0F00DF2E000C0301400000014043FF0080DC
:406B0000080201400803014042FF00800403014041FF00800003014040FF00801402014005FF00801002014004FF008002FF00800402014001FF00800002014000FF008037
:406B40000C02014003FF008028000340000101406000002000001040B8235B004343144A70B5D218150013005A355B33FF35FF3329781E78B14219D24B1C5418DBB2393411
:406B80002B70FF3424789E4201D8A3B207E0D318023139332970FF331B781B0223435C30044A800083500220FFF7E3FD70BDC0460403002000000A4070B5D024124DE400E6
:406BC00029510A200E00FFF7D4FDD22202239200AB500832AA581A4214D0002E12DBC1239B00EB582A595B079B0F120408D4012B08D1D32202219200AB580B43AB5001E0C0
:406C0000022BF6D070BDC04600000A40F7B5060007F0B7FD2E4B00909A5D0193002A53D1A8272C4CFF00E3595B0007D5A823DB00E35828499B0F284815D131E00222274BF3
:406C40001720E358264D1343244AA350FEF790F9013DADB2002DE9D0E359002BE6DB0120FFF787FDF4E70B58DB070AD51D4B1E4DCA587F234F591A401C4BD2033B401A4308
:406C80004A512358134ADB050AD5164B164DD158174BC90A57591940164B3B4019435151C021A82200230906D2002350A15003210A4AA2588A4309496250012201998A55AB
:406CC0000D4A93550D4A9355009807F05EFDF7BD7806002000000A404C20000050200000C509000054200000F4080000FF7FC0FFE07F00001F80FFFF790600207A060020FE
:406D000070B507F03EFD8021D6240C4B0C4A090699501022E400195991431951E424A4001D590849294019516034195991431951FA2189005A5007F028FD70BD00000A408B
:406D4000E407000008FCFFFF10B507F01AFD8021F6220C4B0906D2009950F03A99589950E52189005C58084A2240FC245A502021A4001A598A431A51FA229200995007F096
:406D800004FD10BD00000A4008FCFFFFF8B5304B0E001B78642158431700962408F008F9A400A04208D804000A2801D20A2406E08C2804D99F2805D90325232004E01C25BD
:406DC000962001E018257D20002E00D03570002F3CD060430A2108F0EBF80600952C02D8C820001B12E03220C72C0FD92C23FF339C4205D80A21200008F0DAF8462304E03A
:406E00001421200008F0D4F83723181A10231D4204D1104B1B7858430F4B03E00F4B1B7858430F4B1B785A1E9341DBB2002B00D040420C49081A704308F0BAF8822800DA5D
:406E4000822082380A2108F03DF93870F8BDC04684000020A1F2FF0FA0F2FF0FA3F2FF0FA2F2FF0F50C30000F7B50D00060007F088FC0400B82040007043324B18186B4656
:406E8000FC309E1D0566D91D32002800FFF77EFF2D4B1B78002B0ED02C4B0A211878053008F010F92A4B1A783378002A01D01B1800E01B1A3370D825264BED005959264A2C
:406EC0001F2011403278E8261204F6009F590A4322490F4069460731097801404901394399515A511E4D5A59D2071CD41D4A842690890F221C4950435A581C4F32435A50C5
:406F00001B491C4A5E5880B232405A505E585A58324307261643021CB84200D93A1C92B2520132435A50F021C9005A582000520052085A5001215A590A435A5107F025FC3C
:406F4000F7BDC046040300207B060020ABF2FF0FAAF2FF0F00000A40FFFF00FF1FFCFFFFF408000068060020F8080000FF0100003020000010C0FFFFF8B5B82305005B004A
:406F80006B430F48C41826005B36FF36327000265A34FF3426700B4CAE003619776C0A4C39333C4057033C43FF337464181808F0A1F9002D02D12800FFF7CEFDF8BDC04627
:406FC00004030020FC000A40FF1FFCFF002801D0064A00E0064AA520064BC000195891431950A421C90000205A507047022022220110111100000A40164A830070B59C1860
:40700000154A05009B18154A0A205A66FFF7B1FBA422104BD200002D01D1114900E01149A5209950104AC000AA401958FC340A431A50B8235B006B4318000C4B80221B1896
:4070400000205933FF331870636E12061343636670BDC04600000A40FC000A404A43052001101111022022220010100104030020B82330B50024C0215B0043430C4A490007
:40708000D318FC330B4A9C6383009B185D580A4A2A405A501123A7258340064AED005159200099435151A621C900535030BDC0460403002000000A40FFFEFFFFF0B583000D
:4070C000174E184A184C4000184D002911D1E0279B18FF00D9590E40DE510126370087401159B94311518E215751C9005A58B24312E00C495B18E221C9005F583E405E5030
:4071000002211659814030008843105151518E21C9005858064A024000205A50F0BDC046FFFFEFFF00000A409C04000094040000FFFEFFFFE022074B8000C018D200815807
:40714000054B0B408350E2232022DB00C25000207047C04600000A4001E0FFFF0449054BCA58C8584004830D9002400E181A704700000A40F408000030B50D490D4C0E4BB8
:4071800062581A40002807DB0C4B45012B4013430822002808D108E010231A43FE2340429B03C003184003001343635030BDC046F408000000000A400700C0FFE07F0000EA
:4071C000F7B5070007F0B4FC03006F331E7821331B8801AC2380030072331A780500002A04D0244A11680622114240D12A0067321278012A0DD1951BE9B200223800FFF712
:40720000BFFA0022605531003800FFF7B9FAA0552DE01B78DBB2002B16D0A35D012B05D9012231003800FFF7ABFAA055A35D012B05D8002231003800FFF7A2FAA055002216
:4072400070352B78E25412E01D00EEB2002231003800FFF795FA6055002805D0012231003800FFF78DFA60550135022DEDD12088FEBDC046A4000A40C02210B50948D2001D
:40728000835804001000002904D1074A13408022520303E0054A1340802292031343235010BDC04600000A40FFFFBFFFFFFF7FFF70B500282ED1C2201425174CC000235867
:4072C000AB432350154B164DD65C1038154B00290AD16E60022A10D020580340900603431A0000290ED00FE0AE60022AF4D122581340C02212051A4306E0C021225809059A
:407300001A400A43822300E08423DB051A43C023DB00E25070BDC04600000A4088F2FF0F00FF0A40FFFFFFF3C12108200B4BC9005A5882435A50C022D200995802304900A5
:4073400049089950995801439950985804490140F0200004014399507047C04600000A40FFFFFFBFF8B500250E490F4B01394A1C14D000221F685C689E68A018B24203D03A
:40738000B858A0500432F8E70200DE68141AA64201D020C2FAE710330139E8E707F084FFFBF76AFD0100000088F5000070234343034A4000D3181A8E024BC35AD0187047E7
:4073C000880400208004002010B50022042107F03DFB10BDF0B587B0040007F0BFFA030075331B78002B12D05C233F22FF33C35C93431A32FF32C02B05D1855C05206D069C
:407400006D0E454315E0855AAD05AD0D11E08378804A9B009D581C22130063437E495A5C002A06D0062A04D0CB185B899D4200D21D007A4A63009D52F0236343784AD3183A
:40744000A83302931B789B077CD570236343754AD3184B331B78002B74D173487349A200505004AA971DD61D3B7033705A2D00D25A2501212000FAF749FE4078642140B2D5
:40748000684307F01FFE6A4B4019984200D969483A003100FFF77AFC01212000FAF736FE3B7885783678019307F06BF90322624BE8211A556A46614B1279614F1A55614B14
:4074C0001F221E5510233B555F4B03901D555F4DC9006B5816409343F0221E436E50D200AB5890395B005B08AB506A58584B0A201340019A12021343FC226B500121D200C6
:40750000AB580B43AB50AB588B40CB40AB50FFF730F9E32189006B589B0A9B026B503B5D6A5858010523134303436B50FA230821FC229B00E9509200AB580B43AB500398DC
:4075400007F023F9029B1B781B0761D54149424AA300995020000221FAF7D8FD83782025402B02D801335B10DDB207F00AF902223A4B0A21060020001A70FDF751FDF02141
:407580008120324BC9005A58520052085A505131FF315A580243A0205A505A588005D201D20902435A502E4A11782E4A1278323A521803D43F2A02DD3F2200E000223F2437
:4075C00029480168A1430A43284902605A58920A92025A505A58002D06D02548013D02436D012538054000E0142504201543214A5D50214998505A5802435A50443958589F
:407600001E4A02401E4802435A50300007F0BDF807B0F0BD50F40000C8020020E60200200019000088040020492E00006806002025020000260200001B0A0020180A002035
:407640001A0A0020190A00201C0A002000000A40FF00FFFF192E0000280A002076060020A8F2FF0F8400002090FF0A4010200000050400003C20000044200000FFFFFDFFA9
:4076800001000020F7B50D00040007F067F9070007F077F8242201901E21200001F0E8FB3B0087331B78002B66D0A1373B78DEB2002E61D1962120004900FFF78BFE2000FB
:4076C000FAF7BCFE07F05DF80B2107002000FDF7A7FCD221FF202A4BC9005A58520052085A5020315A5882438E3802435A50254A254998580140042099509958014399509B
:40770000224A234998580140A0209950995880040143102099501F491F4A11601F4A204998505A5802435A50443958581D4A02401D4802435A50380007F027F82000FAF79F
:4077400005FF002D18D070236343184F0121FB181A0048321170598E1B8E994203D916702000FAF7BBFE70236343FA22FD501E210F4B200001F000FC019807F006F8F7BDE5
:4077800000000A40DC080000FFFFFFE714200000FFFF1FC0C97300002C0A00203C20000044200000FFFFFDFF0100008088040020112C000010B50C0007F0D0F80C21022C05
:4077C0000CD0032C04D0614261410423591A05E0943003780421012B00D90C31080010BDF0B5F0244443234E2034A419230088331B7885B005005B073AD5702343431E4A0C
:407800008E34D3181B8E029323889B199B7801335B10DBB21A1C202B00D92022D7B206F0B0FF0390280007F099F85C233F22FF33C35C9343C02B0ED1280007F08FF8238890
:407840000122F6185A236421FF33C35CB25659430097012306E023880122F61802230299B25600972800FDF747FC039806F08DFF05B0F0BD0019000088040020F0234343C8
:40788000F0B5584A85B0D318A8331B780500DB0700D4A4E070234343534AD3181C8E06F070FF002103902800FAF730FC837801335B10DBB21A1C202B00D920220127D3B29B
:4078C00001934A4BC7575A1952781E00022A03D101212800FDF7A4FB022273195A704449444AAB00995038000121434A60439950633107F0E7FB414B0419A0B2404C98429F
:4079000011D8404B984203D93F4B98420CD800E03E48052107F04CFBC5224021D200A35880B20B430BE018000A237D21584307F0C9FBC5224021D200A35880B28B43D42742
:40794000A350FF00E3590A211B021B0AC838029307F02EFB029B00061843E05101272C4A0A20A3583B43A350A358BB40FB40A350FEF7FFFEE1239B00E258BA43E250E258FC
:40798000244B1340019A002A08D0F821224A89001343019A013A52010A4000E01022E121134389006350FA2302209B00E0506C3163587519034363506D78114A85420BD11F
:4079C000802080011158154B154C0B4001210B431159294311511350039806F0D6FE05B0F0BDC046001900008804002076060020792B0000240A0020200A0020D85900004B
:407A000000000A406F1700002823000070170000D407000001F8FFFF05040000FFFFFDFF04200000F023434370B5214A0400D318A8331B789B073AD506F0A3FE0500FC20BC
:407A400008211C4B80001A588A431A50FA2292009950FC220120D20099588143802099509958000601439950D621C9005858124A02405A50E32189005858104A02405A5008
:407A80000F4B1A5D1E00022A03D103212000FDF7C7FA335D032B03D11921200001F048FA280006F072FE0022064BA400E25070BD0019000000000A40FF00FFFF08FCFFFF59
:407AC0001B0A002068060020702343435D4AF0B5D318002285B04533050001911A70904201D1FDF775FA06F04CFE0B2102902800FDF796FAC021544C544B4905E258544F77
:407B00000A430421E250E258524E8A43E250524A524BA1580B40A3501022E251A35993430022A3514E4B02981A6006F02EFE019B03973700002B02D02800FAF77FFC280016
:407B4000FDF786FC280001F0B5FEF02301266B43444AD318A83301931B78334239D006F010FE414B02905B195B78022B03D131002800FDF755FA01213C4BE2588A4380218B
:407B8000E250E25809060A43E250E1229200A158374B0B40FC21A35002228900635893436350FA239B00E250C5224021D200A3580B43C821A3507832A358C9051B021B0A91
:407BC0000B430021A3502B4AAB000298995006F0DCFD2800FDF754FA2800FFF723FF019B1B781B0729D506F0CCFD0422E359C0219343E351039BC905E2508D221201A35851
:407C00000600DB01DB090B438021A350A3588B43A350194A194BA1580B40A350124B1B78022B03D10A212800FDF7FAF9300006F0ACFD0021124AAB0099502800FAF706FABE
:407C400005B0F0BD8804002000000A40DC0800003C2000004420000014200000FFFF1FC02C0A00200019000076060020D407000008F8FFFF240A00201020000008FCFFFF93
:407C8000280A0020F7B504000F0006F07AFD1E2124220190200001F0EBF82000FAF7D6F92000FDF7EDF970236343264E2649F3185B8E8B420CD805222000FAF72BF9011E26
:407CC00006D12000FFF700FF1420FEF752FD0EE07025654375192A8E6B8E9A4203D0200006F064F8688618492000FAF7A9FA7025C8226543920073195A86002F19D0200035
:407D000006F02CFE87300378002B12D02000FAF7E5FB962277510D4D92002B002121200001F02AF92B0001222221200001F024F903E001212000FFF7C7FE019806F025FD96
:407D4000F7BDC0468804002088130000112C0000F0B50B7889B00293AC235B0043430E004E490792CA18039010000025FC3045650298022800D98FE04D32FF321278012AF0
:407D800000D189E003244443E318CC18A379444FDBB2069363792A000593802300979B012900300003F0EEFA0497A84200D0A571AC24039964006143384D72796B18120794
:407DC0004133520FFF331A7003230298D7B25843411869188979002902D00599B9425BD0029930004B4303994C4301211B19EB185A7100229971049B11000093202303F026
:407E0000C1FA002805D02C194434FF342378012B42D0029B013B012B13D8049B002200930721204B300003F0ADFA002834D11C4B0122009307211C4B300003F0A3FA00285F
:407E40002AD1AC24039D64006543144F6A467D192B00127A4233FF331A70049B00220093802311009B01300003F08CFAFC350223002800D140236B65079B002B0CD1029AE5
:407E800003335343039A54431C196B461B7E3F19BB716B461B7D7B7109B0F0BD0C050020FFFF0000F7FFFEFFFF7FFFFF10B50400081F03282FD807F071F8022A1E15AC23D6
:407EC0005B006343144AD3184433FF331B78012B21D1200004F010F900281CD1200006F0C1F818E0AC235B0063430B4A20219B58200098470FE0AC235B006343064AD31893
:407F0000190000225531FF31FC330A705A652021200004F0A3F810BD0C050020F0B5A04F8FB0002801D000F082FC20229D499E4C9E4B0A601C609E4B9E4C1A601C3A0A60D2
:407F40009D490C6080211A603B6809060B439B493B607B5813437B50FAF7CAF8437D012B11D0002B07D0022B16D19022FC211201BB5889030EE090221201B958904B0B4020
:407F80008021490206E090221201B9588C4B0B40F02149030B43BB50C022D200BB5808215B005B08BB50C1230125DB00FA5864208A43FA50FA58834C2A43FA50FEF7D9FB15
:407FC00010223B68182113433B60D223DB00FA588C46AA40EA40FA50FA580A43FA503A5914390A433A51784AB858784A024080200003024374483A507548764A3E58324006
:40800000E026360132433A5080203A59400502433A51E822E026D200B858B6053043C026B850B85836063043B8500220FA586A4E0243FA50F222D200BB587A3083430B4375
:40804000BB50664ABB58834380200B43BB50BA59634BC0011A400243BA518A221201BE5833401843D023B8505E4ADB00FA505E4B00201A00FF325075FA22FE33D2001A8347
:408080005A4B5B4E1D7058709870634633600C33F3607361B161C0210132FF32BB58C905DB01DB090B43BB50BB581D43BD50FAF71FF8431DDB7F0193831DDB7F03930300B9
:4080C0000833DB7F0493030028331B780793C31DDB7F05949AB23C4C02969446FF2B01D1438F9C464349444A7858072502407A50062278582A4B9043019A520002433F48E5
:408100007A503A58920192092A433A503C483D4AB85008203A5902433A51FF24029A906E394AA0431278394C024302988266384AB8582043374CB8503D5937482840374DA6
:408140002843385129480091C67806943448354C354D3649002E6FD0354E9E593040C02676003043324E985198593C26B043183E30432F4E98519858044090208002044382
:408180009C5058590140A020C00301435951985828490140C02080030143995064E0C04600000A4080E100E03DD500005400002000E100E0B9E30000480000200409000011
:4081C000FFFFC0FFF4080000F8080000FFFF0080FC080000FFF0FFFF9C08000094070000FF03F0FF00020080040300207806002000FF0A4064200000E0FFFF7FDC080000D2
:4082000048600000E4080000AEF2FF0F7F100000D4080000782000000100F8FF0B6408013FFCFFFFFF3FFCFFD8080000FFFF0FFF94200000FFFFC3FFB64E9E5930408026A6
:4082400076003043B34E985198593C26B0432C3E3043B04E9851985804409C505A591140C022920311435951C022F8217B5992021343A94A7B51BB5849030B431F211820EB
:40828000BB50A64A82261368B6018B4303431360A34A113813688B4303390B431360A14AA14BB9580B40F821C9020B43FF21BB50BB588B430343BB509C4A9D48BB588B4378
:4082C000F0390B43BB50B9589A4B0B40A02149020B43BB50984A994BB9580B40F02109030B43BB50964A9749BB580B43BB50614606F0E8FE039904008D4806F0E3FEC00201
:408300000443F820904B0002FC50BC590499640C64040443864806F0D5FE8C4A0443BC51B9588B4B0B40802149050B43BB50019B0499022B00D103997D4806F039FE079B42
:4083400064214343180006F033FE824E824ABC598249E40AE4022043B8517B591B0B1B0313437F4A7B51BB585B0D5B050B43BB507C4A7D49BB585B0B5B030B43BB50019B68
:40838000002B24D0794B7A4A9A587A4B1340019A022A01D0C02216E00022774D691C8E784C78360624042643AC5C900826430C78043224023443714E0431801980003C50A1
:4083C000202AECD1E02252031343694ABB508022674B5205FB58FF211B011B091343644ABB504C4B664AFB5813434A4ABB50BB5801229343474ABB50624A13680B4204D11E
:4084000013688B437B390B4313605F4A5F4BB95800200B40802149000B43BB50B9585C4B524C0B40802109050B43BB50F9F760FE437F002B62D0837F564E9C46C37F0193F8
:40844000831CDB7F027F0393534BE1587F230B40A1590491411CCD7F29040791049D4F492940079D29434E4DA15166594D4931409C26360231436151474D032A05D9027FE6
:40848000043AD2B2062A00D906228E203A4C52000001A2183958128C89B2120411433950FF20029AD16E404A814312781143029AD1666246012A07D0002A03D0022A05D189
:4084C0003A4A02E03A4A00E03A4A1343019A012A04D0022A05D1FF22120201E08822D2011343039A002A01D18032134380227B51069BD204FB581343069ABB502E4B2F4A87
:408500009B6C93425ED02E4A9B18012B5AD9FEF795F9FEE7942000002820000084FF0A4088FF0A40A0200000FF3FC0FFA4200000C05D0000FF3FF0FFA8200000FF0FE0FF25
:408540007C200000000010508420000070200000FFFFFF807420000046020000FF040000882000008C200000FA04000000000A4090200000FFFF0FFC5CF40000040C0000BA
:408580000000F01F68FF0A409C200000FFC0FFFFFFFFFF8168200000EC080000FFFF80FF6C2000003F00FEFFADF2FF0F0000FF100000101000003410FCF0FF0F012B0000FD
:4085C000FAD4FFFF002306220A21012000F008FE02225520059B4042FB58FA261343059A3601BB50FEF7C8FD05250024002005F02FFC82B2031CA24200D2231C013D9CB2A1
:40860000002DF3D1B04204D8FA23241A5B009C42EADD8F4B08A91A00303251CA51C10BAE32003C3313CB13C200228A4B1A710293009B6420FA58884B884C1A4008AB5B59EF
:408640000193990273595B010B431343009ABB50A8220023D200BB508022009B1206FB581343009ABB50FEF784F8A823DB00FB58DB054CD57A4AA3589B03DB0D47D0794D60
:40868000A058A258635980035201D20DC00DDB058018DB0DC018744B0321E65806F088FC724B80B21E4043021E436F4B0430E6506F4B0005E2586F4B134018436C4B6E4AD0
:4086C000E0506E4B6E48E158694BC90AE35801401A400B001343664A6A49A350635860589B034001DA0DC00D8318605903218003C00DC0185C4BE55806F05AFC6D0A5A4B9C
:408700006D022843E0500123029A13711DE0A8230022DB00FA500A20FEF72BF880225A4C12062368C82013432360009B009AFB5804355B005B08BB50FEF71BF823685B0076
:408740005B0823600C2D00D072E7002005F0CAFD4E4A4F4D13684F4C0533136006F011F820223C4E4C4B0090B3607B59012113437B51D423DB00FA58484B0A201340E0228D
:40878000D2001343603ABB50454ABB580B43BB50BB588B40CB40BB50FDF7EBFF85220121D200BB588B43BB50BB58F5318B43CB390B43BB5004223B4BFA503B5913433B51C8
:4087C000009805F0E2FF05F0DCFF8022364B0090F3607B59012113437B51D423DB00FB587F329343543A1343D422D200BB504932FF32BB580A200B43BB50BB588B40CB408F
:40880000BB50FDF7B6FF0121284ABB588B43BB50BB58F5318B43D1390B43BB500222214BFA503B5913433B51009805F0AEFFC023DB00F9581E4A0A40FA50FA58FA50AA229D
:408840009200B9581B4B0B40BB500FB0F0BDC0465CF40000780600201F00FCFF00000A40B4200000BC20000090200000FF01FCFF94200000FFFF0FE0FF07F0FFAC20000018
:4088800000F80F00B8200000DC000A4080FF0A40CC0800004C0400007D690000FF00FFFFEC070000440400008968000024040000FFFFF1CFFEFBFFFF70B505000220002D61
:4088C0001FD144200F4CFF30265C3538FF38012E17D05620FF30205CA22040002154A52149006254072213404C22FF32A354A3235B00E55202332800E554049903F01AFC5B
:40890000280070BD0C05002070B504000D0006F00FF9030001226E3383301A7010210570200000F005FB2000202106F019FB0221200006F009FB70BDF8B504000D1E05D13C
:4089400005F02AFC954B0F2205215CE001290CD1052100F0EDFA200003F0CEFB002800D01AE1200005F07EFB16E1022903D105F013FC202104E0032906D105F00DFC0821BF
:40898000200003F06BFB07E1042917D1AC235B0043438349CA184532FF321578052D0AD1072100F0ABFA002800D1F5E02900200005F084FAF0E05B581021EBE0052903D1D9
:4089C000072100F0B5FADAE7062920D105F0E4FBAC235B006343724A0421D31801225533FF331A702000043200F042FAB821490061436C4B0022C91804312000FFF7A8F90A
:408A000003222900654B200000F0B6FAC4E007295FD1062100F08CFAAC235B006343604DEB185533FF331B78002B09D0B821490061435C4B0122C91804312000FFF788F9C9
:408A4000AC235B006343EB181A004432FF321278012A16D11A004532FF321278022A10D8FC335B6D002B04D01021200003F0F6FA07E0200003F040FB002802D1200005F0F7
:408A8000F1FAAC277F006743EE1933005533FF331B78002B14D0FC36736D002B10D0B821490061433F4BE819C91804313430432200F0C2F9EB59716D200098470023736525
:408AC000AC235B005C4300232D195535FF352B7062E008292DD1AC235B001A004243304DAA185632FF321278002A05D01A004243AA185832FF3212786343EB181A0056323F
:408B0000FF321278002A02D05733FF331B781021200003F0A3FAAC235B006343EA18100000215532FC30FF324165EB581170013130E0092916D1102103F090FA06212000AD
:408B400000F0F6F9AC235B00634315490020CA1815005B5880215532FC35FF326865C901107017E00A2917D1102103F077FA0621200000F0DDF9AC235B0063430849002088
:408B8000CA1815005B5880215532FC35FF3268650902107020009847F8BDC046AD7E00000C05002004030020704700000C2359436933FF334343C9180C4B0D4A5918FF23F4
:408BC0008B72135C013BDBB213540A4A1378013BDBB213701378002B06D1074B1B78002B02D10822054B1A607047C0463C010020B0020020B10200208806002080E100E09C
:408C000010B5024B5988F9F71BFB10BD8806002070B504000D00F9F76BFA0530C67F200005F09CFE022E22D172300378002B1ED0114B1B78052B1AD1702363430F4AD3182C
:408C40001B8EAB4213D2FA22EB1A520093420EDD0B4B0C4AD3585B019B0E08D00A4B0B4A012120005D80FCF753FC002803D029002000F9F7E5FA70BDF00200208804002089
:408C8000B020000000000A4088060020018C000010B572B6044A054B11685B680B431360FDF7CCFD10BDC046600000208806002070B5074D074A2B6811889BB204001600BC
:408CC0008B4202D06420FDF754FD2C60348070BD40000340EC0200200123F7B53C4E3D4D73642B700096009BDC6B2B89A2B29BB22404240C9A4202D880214902641800274E
:408D0000E41AA4B22A81344ABB18997A0192C9B2FF2920D01868621D904202D91A68121B00E000221A601868002814D1FF229A722A4A944666461278013AD2B23270284AC2
:408D4000944666461278013AD2B232705A68002A01D05B689847BA230C375B009F42D2D11F4C2378DBB2002B1ED000231D48019AD218917AFF2903D01168814200D21068DF
:408D8000BA220C3352009342F1D1009A2B89D26B9BB291B21204120C8B4202D3802149025218D31A9BB200E00E48053383429AD880B268812B89C01880B2FFF779FF00231F
:408DC0002B702378002B02D10822074B1A60F7BD00000340880600203C010020B0020020B1020020C0FF000080E100E0F0235843014B2030C01870470019000000487047B1
:408E00000019000070B504000D0005F0BAFC002C02D02368AB43236005F0B7FC70BD70B504000D0005F0ADFC002C02D023681D43256005F0AAFC70BD002310B59200934210
:408E400003D0CC58C4500433F9E710BD031E0CD00023994209D04118814204D0027801309B18DBB2F8E75B42DBB2180070470000F7B505000F00009205F083FCBA230600D3
:408E800000245B006B4301930C236343019AE1B29B18094AD3189B7ADBB2BB4205D3009A934202D82800FFF781FE01341F2CEBD1300005F06AFCF7BD3C010020BA2370B5C6
:408EC0000C265B0058430C4D91420DD8FF290FD00024330063431B18EB189B7A994205D001341F2CF5D103E0002004E0012002E00131C9B2E8E770BD3C01002030B50023FC
:408F0000FF2911D0BA220C2552005043074C2A005A431218A218927A914204D001331F2BF5D1002300E00123180030BD3C010020F8B504000D0005F024FC0600FF2D11D0D2
:408F40000C22BA200023944640006043094F62465A431218BA18927AD9B2954206D001331F2BF4D1300005F010FCF8BD2000FFF71DFEF7E73C010020F0B585B005000F00A9
:408F8000160002930020FF297AD0824278D0BA235B006B433B4A9B18019305F0F2FBFF231E22019903906931FF31887AFF2800D1D3B2887A87420BD13349D3B24A5D013A72
:408FC000D2B24A5531490A78013AD2B20A7007E0013A52B20C39501CE7D10024FF2B4BD00C225343019A2A49D318029A1E815A60284A9F721288254C56431E600A78002A1E
:4090000030D1254AD26B207897B200281BD00E891204B6B2120CBE4202D3802040021218921B1E6892B292191A6018684A89904218D21B689BB24B8108894B89C01880B2C5
:40904000FFF736FE0EE00F811868144B984200D9180080B2C7194881B8B2FFF729FE08220F4B1A60084A535D0133DBB2535523780133DBB223700124039805F086FB20008E
:4090800005B0F0BD3C010020B0020020B1020020880600207406002000000340C0FF000000E100E010B50023FFF766FF10BD000010B50D4B1A6801321A601B68012B0BD952
:4090C0000A4B1B68002B02D0002108009847084A084B5A60FDF7B2FB074B084AC2210020FFF74AFF10BDC046E8020020700600200C3003C0000D0020B1900000EE020000DD
:40910000C82110B5002289000400F8F703FF002805D12000FEF708F9FA22520009E0702308216343064AD31842331A780A431A706422044B2E212000FFF71EFF10BDC046D1
:409140008804002049910000C82170B5002289000400F8F7DFFE002824D1702308216343144AD31842331D780D4008D01A7820008A431A70FEF7D8F8FA22520013E07F2219
:40918000197820000A401A7005F068FE29002000FEF772F820000121FEF76EF8200005F05DFB05E06422044B2E212000FFF7E4FE70BDC0468804002049910000064B1B7B7C
:4091C0005B0706D4054B58680002000CC001803001E0C0204001704788060020C0FF000070B50F24012520400F4C002B04D0854023681D43256003E085402368AB4323606D
:409200000323072643439E409A40A5688000B5432A43A2600F2282408140044C236893431943216070BDC04600000440000002400D4B70B504000625984212D84378027809
:409240000A491B0213438B420BD1C1798379090219430A390A30FFF7F9FD237A834200D10025280070BDC046FFFF000059430000F7B504000D002D4F2D4E022904D0062350
:40928000019305290FD001E007230193200005F0D9FD012D07D170236343264AD3184B331B78002B11D1200004F0C4FC50280CD909236343FA18525DFF2A06D032000D3297
:4092C000D3185A5D0132D2B25A55092363430D36F618FF18725D7B5D200093420DDB05F0A7FD0199200005F0EDFD00281CD000220421200005F0AAFB16E005F02FFB030049
:4093000072331B78002B03D067300378002B08D1702302216343074AD31842331A780A431A70200005F062FDF7BDC046300100208806002088040020F7B5154B154C197894
:40934000154D164B164E1F7822782B783F020193337839439C46019B00B21B02134362469B1ACF1A0F4B1421C01805F0ABFE24782D783678EDB22D02E4B2F6B22C430A494B
:40938000A41B78434C43001905F09CFE00B2FEBD91F2FF0F8EF2FF0F8FF2FF0F92F2FF0F90F2FF0F78ECFFFFEE020000F0B5D04E8BB00190CF4D3078EC8A042800D948E275
:4093C00005F0B4FF050066008D014702DA012E8B1421A31B1BB2DA179B1853402000029305F070FE029B834206D81C23019A5343C14A9B5C032B40D1AB7E002B3DD1BF4A84
:40940000BF491378DBB28C4203D92000FFF794FF26E012786421002A00D019B2B948BA4FBA4D3B782A7806783F781202FFB2039713432D780778B6489E1B7618001B1421D6
:4094400005F040FE6421039BEDB22D021D43FFB24942EF1B4F437043C01905F033FE00B2A44B0299DA8B801AFA229883520091420CDCF43AFF3A9A7608E020B236B2801BAB
:40948000142105F01FFE0123A883AB76994B1C830022984B987ED91CCA771A849449904203D004209A76087001E002220A70D98B9A8B01988A1894B222B207926A46928B92
:4094C0009449DA83019B944A9B009950F8F710FE059005F056F918220026904F904B0990FB58934304938F4BFA588F4B1A4015008E4B019A9E548E4B9E54FDF72FFE894B50
:4095000002900693079B0397B34222DBB0420CDA1023049A01991A430492844A0F3B47421D435354BFB2330002E06B4637001B8922001A4300D19AE1082204990198114363
:4095400004910121F8321543794A11540022069222E0029B002B0DDD08226B460499019811430491F83272491543FF3A1B890A54370003E0029B5F423300BFB2624292B2C6
:409580000692102204990024114304910121694A01981543654A1154079A02998A4220DD022280269543B6002E430894A34202D001339BB20893069B9F4201D0013FBFB21C
:4095C0001825059B188B6843013880B2FBF7D0FC029B002B26DA059BD88E1EE01400130006920222544E08942E401643A34202D0013B9BB20893069BBB4201D00137BFB270
:409600001825059B588B6843013880B2FBF7B0FC029B002B06DC059B188F4543013DA8B2FBF7A6FC069B1A02FE23DB011A407F231F401743414B039AD750414B220413404D
:40964000089A9405A40D1C43039A3E4BD450019A364B9B5C002B16D0354B9B5C002B12D0079B029A934207DD059BDA8E1B8B9A4209D0354B1E4006E0059B1A8F5B8B9A4284
:4096800001D001239E43039B0499254A012499500321039B234A9E50039A2C4BD2588A430399CA50C021A82203980906D2008150A9218020039AC9005258C0050243039827
:4096C000425000210198224A1154039A0399D2582243CA50099805F058F82300BAE0019804F064FB2B8C984234D21B1A33E0C046F002002088060020C8020020A6F2FF0FA7
:409700008713000090F2FF0F8EF2FF0F8FF2FF0F88130000B5A600000C0A002000000A40F40800004C200000FEFEFEFF790600207A06002001000100FFFDFFFF5820000058
:409740000000FF035C200000FFFEFFFF5020000078060020C31A1BB2C82B04DD002328840335EB7776E00335EB7F0133DBB2EB77132B6ED904236BE01E210198FFF7BEFBE2
:40978000002864D07023019A434F5343FB181A004B321278002A37D004F0F3FFBA210022019B4900594304003C480C2353435B18C718BF7A1E2F04D001321F2AF5D10025CE
:4097C00014E018582B899AB2354BDB6B99B21B048A425AD21B0C9B1A9BB20025984205D9C01A304B198805F0E3FB0500200004F0CCFFFA22521B92B20E2A01D9052221E023
:4098000014239A1A92B21DE048331B78002B08D17023019A5343FF1848373B78002B18D108E01422210052420198F8F773FB0028E4D1EDE7E98A14220198F8F76BFB002890
:4098400007D1DBE7184B20210198FFF795FB052333700023154A1278052A1BD0002B19D1134B012257210198FFF786FB12E0079B02998B4200DCB1E6022380269D43B600AC
:409880002E4314000692089295E680211B0C49025B18A0E70BB0F0BD880400203C0100200000034074060020112C0000F0020020AD93000070B557210500FFF739FB0B4C69
:4098C0002378052B02D02800FDF7A0F90849094A094B885803408B50084B094A05211A83002204335A832170DA7770BDF002002000000A40F40800000500C0FF88060020A8
:4099000088130000022906D1002804D1A623024A01395B00D15470470C05002010B5092902D1023101F02EFF10BD0000F8B5040005F0FEF893239B0063431D4D1D4AEE1884
:40994000B61832780700002A0FD102005B5999329B7A2000DB09137005F0EAF801233370030099331B7898300370932392229B0063439200EE18B6183278002A17D1EB58F6
:4099800097371B7920009B093B7005F0D1F83378002B0CD1013333700300943097331B7802789A4200D90370200002F01BFEF8BDB00600204902000010B5022905D1C82217
:4099C0000731920001F0D6FC04E0082902D1043901F0D8FE10BD0000F8B50D00040005F0A7F80700A81E08286AD805F0D7FA051855555569696959002000FFF797FF9323B8
:409A00009B0063432F4A20009A583B009168FC339964C0373B682C4ADB6A984750E09325AD006543274A294B5519EB181B781600032B04D10E21200001F0A4FE40E03A004B
:409A40008F23FC32926C9B00EB181A60902275373B789200AD18002B02D10821297006E0200005F09FF9002805D117212870200001F088FE04E0042320002B7001F0DFFE3C
:409A800093228F23920062439B00B218D2181621200005F009FA13E0200001F097FE0FE093239B006343074A0849D3181A008532FF3212785B181A700021200002F04CFD59
:409AC000F8BDC046B0060020C5B100002202000070B50D00040005F02BF8022D1AD101237A3003700021200004F038FA8022124D52032B68322013432B60FCF73AFE802242
:409B00002B68520213432B6037220921200001F031FC10E0082D0ED1074B084A19687A300A401A601968064A0A401A6000230370200001F06BFE70BDC4000A40FFFFFEFF2A
:409B4000FFFFEFFF10B5040004F0F2FF93239B006343114AD318114A9B181B78092B02D00B2B0FD017E0663002780D4B002A01D1013200E00022027020001A5502F032FDA0
:409B8000162105E07D3003781321012B00D01221200001F0F7FD10BDB006002047020000EC0B0020F8B50F00040004F0C1FF93239B00010018006043424D434A2818801881
:409BC0000678B81E08287BD805F0E8F905315252527A7A7A56000B003000C03309381B680A286DD805F0DAF906080D6C6C6C6C6C6C6C0F001B6B00E05B6B344920009847D1
:409C00005EE09B6BF9E79322920062439431AD180B788535FF35012B01D9102300E0042380212B70C900200005F076F948E06343274AEB189B181B78032B15D00D210A2E4F
:409C400004D00B3E711E8E410F23991B9322920062431F4BAA182000D21805F025F91721200001F08FFD2BE02000FFF76BFF27E0200001F0ABFD23E06343EA1811008531BC
:409C8000FF311348097812181170092E07D1012905D1EB181A180D31200005F005F99322920062430A4BAD18ED182A78012A03D1200001F0C4FD03E00021200002F04CFC7C
:409CC000F8BDC046B006002047020000C5B100002202000010B50400881E04281AD805F05DF9030D161616000021200002F068FC03220021200002F02FFC0BE0200004217C
:409D0000FCF732FD0B21200001F03CFD02E0200001F095FD10BD000010B50400881E06284ED805F03BF904122F31334D42002000402105F0FDF80021200002F041FC0D220B
:409D40000021200002F008FC3AE0932391209B0063431C491A008000CB181B180020187091238A189B00D2182000132105F09CF820000321FCF7F8FC1B220921200001F0D2
:409D8000F9FA1DE0002115E0012113E00821200001F09AFB002810D020000421FCF7E4FC0B21200001F0EEFC0AE01021200005F06DF802212000FCF7D7FC200001F03FFD87
:409DC00010BDC046B006002037B50400881E062828D805F0E3F8040E1414162714000121200002F0EDFB0D220121200002F0B4FB18E01B220921200001F0BCFA12E00B2129
:409E00000DE09320002280006043074D009201210823405901F0B6FA414241410A31200001F0B0FC37BDC046B0060020F0B585B00400019104F07CFE037C93250293030056
:409E400079331B78AD006543DBB203935D4B019A5D195D4B0600EB181F78022A00D08AE0200004F065FE020000239B3213702D3A1370564A0121AA181370554AAA18137003
:409E8000020081321170013A137081229200AD180200FC322B8093648A22FF3283549C421AD12100200002F08BFB0121200002F087FB0199200002F083FB464B1A00FC32F3
:409EC00054651A005532FF3214701A0044334D32FF32FF3314701C70200002F083FBB8235B0063433C4A3D4DD31800222A33FF331A70A0233A4ADB00EA50200004F018FEA8
:409F0000E022A2239200DB00EA5094300378012B05D980219932FF32AB580B43AB50A123DB00EA582F490A430221EA50EA580A43EA50002F02D03722073107E0029B002B74
:409F400008D0039B002B05D132220921200001F011FA34E03200BE321388002B2BD093239B0063431749CB181F495B180121197012880831EAE7019A082A20D1002F0FD0A9
:409F800000221A70029B0B21934215D0039B934212D103007D331B7893420DD002390BE0114B0A21ED182B78002B05D02F700131200001F0E7FB0B21200001F0E3FB05B03B
:409FC000F0BDC046B00600200302000001020000020200000C0500200403002000000A407F0609040006090446020000F0B585B00E00040004F09CFD03000090FC33B01E34
:40A000009D6C062800D9ABE004F0C8FF048996969EAAA60093239B006343524AD318524A03939B181A78012A06D1002101321970200002F091FA93E06B005B0F4133009A5C
:40A040009B00D3185E683F23370E9F430297C02F26D1464A0A21200001F08CF980212000490204F065FF642233041B0E5A43019214222B035B0D5A43052317003C4A6D0620
:40A0800094466D0E5D43039BF93A63441B78FF3A9343C02B24D10F21200001F073FB24E00A212000FEF744FF80212000490204F03FFF0022009B02999B331A7033039B0DAF
:40A0C000323253430193B3009B0D019F002901D05A4317002B0101D52D0300E0AD05AD0D1C220921200001F045F993239B005C431C4B6A461C198A2392889B00E3181A80C1
:40A100001C4BE3181F8089239B00E3181D808D239B00E418009B2660FC33DE6520E003212000FCF721FB200001F0BEF81C220921200001F01FF913E020000021FCF714FB84
:40A14000200001F043FB0BE020000021FCF70CFB200001F074FB03E00F21200001F012FB05B0F0BDB006002006020000B0360000370200002602000037B50400881E0A286A
:40A1800054D804F00BFF062B39393153535353533900200004F0CCFC030095331A78244B1900012A03D97C3001784903194393229200130063431F48C5182A0001237D32F3
:40A1C000FF3211602000009219000F22FEF774FB194BED182B7801332B7027E01B220121200001F0C7F821E093239B006343114A2000995801F000F901212000FEF798FE31
:40A2000080212000490104F093FE09212000FEF775FE002806D0200004F08AFC0C23A230037003E00B21200001F0ACFA37BDC046018000FFB006002002020000F8B50D00FC
:40A24000040004F075FC0600A81E062800D9B5E004F0A4FE041C85858589980093239B006343574AC036D318564A35689B18198820006B6898472000EB6853499847C822F3
:40A2800009215200200001F075F897E09325AD0065434B4933004D198D21FC339A6C89001A65691809682000D965DA6404F040FC444B0700EB181A880300AE331A808A23E4
:40A2C0009B00EB181A880300B0331A80892302009B00EB181988AC3211800121373A11700E3A1278364D8A4206D119880300C0331B6820009B689847200000F0DFFF20000C
:40A3000002F070F99322920013009021012063438900EB185918FC370870386D8F27BF00DB191860430101D503230B708F2362439B00AD18EA181621200004F0B5FD200031
:40A3400000F054FF8B361721200001F01BFA3378002B33D101212000FBF778FB2EE0200001F06DFA2AE020000921FEF7E1FD80212000490004F0DCFD06220021200002F01B
:40A38000EBF81BE09323902018259B0063430C491A008000CB18181805708F20FC3680001B18B06C8A1818608F239B002000D218162104F079FD200001F07EFAF8BDC0465E
:40A3C000B0060020260200006FB10000F8B504000F0004F0ADFB0300C03305001E68072F23D0082F35D0022F4BD181782000FBF72DFB2B0070331978200073699847002320
:40A4000076352B703621200004F040FD04F0BAFA002824D004F0B6FA09210200200000F0A9FF0122174B1A552BE0200004F080FB020000239A32763013700B21037020007B
:40A4400004F024FD3900200001F09CF90E4A022110E00C4B1A5D002A10D000221A550A492000736898470949F3682000984714220921FF32200000F07DFF02E0200001F02B
:40A480001BFAF8BDAC060020881300006FB1000070B50E00040004F04BFB0500B01E0B2842D804F07BFD0641414127412B414141413EB4220921200000F05CFF2B7C012B6C
:40A4C00032D12B0079331B78002B2DD193239B006343164AD318164A9B181E7804F046FA864221D20A23A2352B700421200004F013FD19E0200001F069F915E093239B0052
:40A5000063430A4AD3180B4A9B181B78312B04D80B21200001F036F906E0200001F0AEF902E0200001F08BF970BDC046B0060020020200000102000073B50E00040004F0A4
:40A54000F7FA0500B01E0B2800D9A0E004F026FD06214253719C8A9F9F9F9F922B0074331B78062B06D1C0352B6849491B69200098478CE0200004F0E3FA2B000D35FF350B
:40A580007E331B780122009500212000FEF794F97DE002212000FEF7CBFC80212000890104F0C6FC012376352B7093239B006343384A2000D31880229200991800220A7010
:40A5C00035495B18F9391A70FF391B3200F0D2FE28212AE02B0075331B78012B0BD193239B0063432B4A1721D3182C4A9B181B78012B2CD132E076352978C9B200292DD134
:40A600009325AD006543234B20005D19224BED182B7801332B7001F0D3FF0C21200001F0B1F82B78062B32D12721200004F02EFC2DE09320012280006043164D00920423FC
:40A640000021405900F09EFE002804D00D21200001F098F81BE02000FFF768F9200001F0B5F814E02000102104F010FC200001F0E6F80CE076352B78002B08D18021200066
:40A68000890104F049FC02E0200001F0F7F873BD6FB10000B0060020010200000A020000704700001C2300225843014BC2547047C802002010B5034B01225721FEF75CFC0F
:40A6C00010BDC046AD93000070B51C244443184B05001C19E37C022B26D90023227E154EE3742376012A13D9FA23E17D9B0009095943114BC918F7F7A3FD0F22E37D3100B5
:40A70000134053434B3363812800FCF7BBFF0BE009492181F7F794FD96235B00638131002800FCF7AFFF02E02800FCF765FC70BDC802002011CC00008813000010B50028CF
:40A7400008D104F00BF977300078C0B2002801D104F0A0F810BD000070B505000C0004F010F81C236B43044AD3185A68A2435A6004F00BF870BDC046C802002070B505002D
:40A780000C0003F0FEFF1C236B43044AD3185A6814435C6003F0F9FF70BDC046C8020020F0B50400481F85B0062800D999E004F0F5FB52116885989804002000FCF706FC58
:40A7C0001C2301216343484A2000D3185970FFF7D5FF86E0B8235B006343444A4933FF33D55C200002ABDD71F7F774FC1C220100C379012062439C463B4B08319A185076A0
:40A800000A00624400920F272A0008003A400192009A904213D02A0006787240BA430CD1019A3E40B24208DC1C2262439B1801225D751A7502ABD91D09E00130E8E71C2209
:40A8400062439B1800221A75DA741A7662462000FCF792FB45E01C2565432000FCF7B6FB214B23495D1929812000F7F7E9FC21492000FCF707FF0023EB742B762B756B76C5
:40A880002CE01C22624318498B181A7D002A0DD0DA7C987D0132DA745A7D904206D11A7E0132D2B21A76022A00D1D8751C2300226343CB185A765A7D9A750BE01C23634302
:40A8C000094AD3185A7E012A08D100225A76DA7C0132DA742000FFF7F7FE02E02000FCF78BFB05B0F0BDC046C8020020040300208813000011CC0000F7B504000D00F7F753
:40A90000E9FB0700042D00D19EE00B2D03D0032D00D0F8E00CE02000FCF7AAFB1C2301216343794A2000D3185970FFF727FFEAE01C236343744E7549F218D2898A4208D033
:40A94000022220009A55FCF793FB10212000FFF703FF1C252B006343F318DB896B4A934202D02000FFF7EAFE812165437219D38949009BB28B4218D00BD8012B10D0022171
:40A98000FF318B4200D0BEE096235B00538160491AE05E498B421FD05E498B420AD0B2E096235B0053815C490EE096235B0053815A4909E002217B798B43012B00D0A2E00C
:40A9C0002C33FF33564953812000F7F739FC55492000FCF757FE96E07B79012B00D892E096235B0053812A3BFF3B73556E33FF3363434D4A8020D3180022FC339A634B4A5D
:40AA0000A3009B18C02252009958400001439950012198580843985098580842FCD1D82149005858424A024042485A5002435A501123A621A340A7203C4AC9005350C000A8
:40AA400011580B4313505EE003F09BFEB8235B006343354DEB18FC339E6B03F096FE0195C825002E07DD70236343334A7543D318198E4D190BE0702363432F4A7142D3189C
:40AA80004D43198E2D4BCB189D4203D84D1B2C4B9D4200D82B4D7B79022B04D11C4B9D4206D91D0004E0032B02D11D4B9D4203D8194B9D4204D900E01D002000FFF73EFE8E
:40AAC000702363431C4AD3181B8EAB420ED01C2363430D4AA9B2D3189622520020005A81F7F7AEFB0F492000FCF7CCFD03F049FEB8235B005C43019B1C19FC34A36B9E1B2F
:40AB0000A66303F042FEF7BDC802002001020000E02E0000020200008813000028230000204E000011CC00000403002000000A4004F006F00105030588040020B8F2FFFF38
:40AB4000470D0000480D000070B504000D00F7F7C1FA03000B2D6DD8280004F01FFA066B6B376B5C486B686B6B305B781B0761D51C236343304AD31800221A75DA741A7699
:40AB80002E4AA30099182E4A9B18586C2D4A02408020400102435A64586D2B4A0240A020400002435A65D8235B00C858274A02408020CA50CA5840020243CA5037E01C23C1
:40ABC000012163431C4AD31859700CE02000FCF7FDF91C221300634317491A3A5A54CB18082105325A702000FFF7C8FD22E01C2304216343104A20009954D31896225200D5
:40AC00005A81253AFF3A5A703C31FFF7B7FD2000FFF794FD0EE02000FCF7D8F91C236343054AD3180022DA741A761A755A762000FCF7E2F970BDC046C802002000000A4074
:40AC4000FC000A40FE1FFCFF01FEFFFFFFFF07F073B504000D00F7F73DFA0600002D02D0012D25D03DE01C2363431E4A0C21D31801221A734078084211D0DA8120001A82D2
:40AC8000FCF758FAE0218820174AA3009B18C9005A58000102435A506420FBF76AFD01230093002320001A001900FAF7B1F818E000212000FCF702FA02212000FFF74CFD36
:40ACC0001C230C22707807496343104203D00622CB185A7001E0CB185D7001212000FFF74DFD73BDC802002000000A40F7B504000D00F7F7EFF90600092D00D9F2E02800F6
:40AD000004F04CF90595AAF0F0F0F0F0F0C000212000FCF7D3F901212000FCF7CFF9472120004A22FEF7A4F8012120004942FFF713FD002C0FD1E02201216B4BD200995040
:40AD40001F311032995080211A6889040A431A603220FBF70EFD02237278644D1A4037D0002C1AD12000FCF7E5F92000FCF7E2F9E02284205C4BD2009958000101430820FE
:40AD800099509958014399501032995838300143995099585648014399501C23327955495200525A01216343EB185A8173780B4205D00091062302222000FAF729F81C2380
:40ADC00001216343EA18917611730522EA541BE01C236343E95C012902D0EA54EB189A762000FCF7A7F9E02184203F4AA3009B18C9005A58000102435A50022200230092AC
:40AE000019002000FAF704F8002C08D020003A49F7F716FA39492000FCF734FC62E0200003F09CFD77300378002BEFD15AE01C23002163432D4A0126D518995496235B00BB
:40AE40006B81AE762000FCF739F9022331006B702000FFF793FC45E01C236343234A9D5C052D3FD101212000FCF728F9012120004942FFF771FC224B2A0047212000FEF75B
:40AE80007BF82FE01C266643184FF35D052B29D1002302220093012106332000F9F7B8FF051E18D12000FCF745F92000FCF742F9E02184200C4AA3009B18C9005A580001D0
:40AEC00002435A500222BB199D761D73F5552B000092290003E001210623022200912000F9F796FFF7BDC04600000A40C802002000040004A4F400008813000011CC00000A
:40AF000013CC00001C2370B543431E4E0400F3185B78002B33D0FCF70DF900212000FCF7CDF84B2247212000FDF7A2FF002C1AD1E2238022144DDB00EC501206103BEA507D
:40AF40000423124A5B42A95820000B40AB5003220F4BEA50FCF78CF82000FCF737F82A680C4B13402B601C2300225C4333195A605A701A739A763255C82292001A810020E6
:40AF800070BDC046C802002000000A409C04000094040000FFFFFFFD37B504000D00F7F799F802000A2D00D9D8E0280003F0F6FF06215CD6D6D6D6D6D68EAF001C2300217E
:40AFC00001256343664A2000D318597302220B000095F9F71DFF02222900009205232000F9F716FF5F4B604A47212000FDF7C4FFB4E01C2363435A4DEB185B7B002B25D155
:40B00000527809331A420BD080212000C900FFF7A3FB544B962248212000FDF7ADFF08E047212000FDF784FF802120008900FFF793FB00230222190020000092F9F7E8FE98
:40B040001C235C431B3B2C19637387E020004821FDF76EFF80212000C900FFF77DFB00212000FCF72BF850E047212000FDF746FF002821D020004721FDF75AFF8021200041
:40B080008900FFF769FB20004821FDF751FF80212000C900FFF760FB00212000FCF70EF820000221FFF758FB01210523009102222000F9F7ADFE51E001212000FBF7FEFF23
:40B0C0001C236343264AD31802221DE000212000FBF7F4FF02212000FFF73EFB01212000FBF7ECFF04212000FFF736FB48212000FDF71EFF80212000C900FFF72DFB1C234B
:40B100006343174AD31805225A70012123E000212000FBF7D3FF02212000FFF71DFB01212000FBF7CBFF04212000FFF715FB47212000FDF7FDFE802120008900FFF70CFBAA
:40B140001C23012163430648C218195496235B001173538151702000FFF710FB37BDC046C802002013CC00004C040000704710B5802103F0D1FE10BD0139CBB210B5002189
:40B18000092B02D8024A9B00995803F0C5FE10BDACF4000010B503F0BFFE10BD93239B00434310B5893304000548FF331818202204F0A0F880212000090103F0ADFE10BD35
:40B1C000B006002093239B00434310B5813304000548FF331818082204F08CF880212000C90003F099FE10BDB0060020F8B5050003F09EFC93239B006B43284E284AF318EC
:40B200009B1800221A70037C0400934235D0030066331B78012B04D0030094331B78012B2BD9230081331B78002B26D023007D331B78002B08D193239B006B43184AF31835
:40B240009B1801221A7018E02700C0373B682800DB699847002810D1230079331B78002B05D02300B9331A7818231A4205D03B68703421785B692800984793239B005D4356
:40B28000483B7619F21800231380064AB218137082229200B6183370F8BDC046B0060020070200000902000010B503F041FC020000238532C4301370036010BD70B5060030
:40B2C00003F036FC0300050075331B7804009535012B04D1030094331B782B7003E0300003F06EFD2870963423782A789A4200D92B7070BD93239B005843044B1818802384
:40B300009B00C018002303707047C046B0060020F7B5060001920D0003F00AFC030085331A78012A23D1C430026807000092032D01D000221A70009B002B18D0019B019A31
:40B34000002B0CD09324A4007443094B24221C193534FF340199200003F0CCFF220029003000009B9847032D01D000233B60F7BDB006002010B5024BFDF7FEFD10BDC046BF
:40B3800079B1000070B504AC2588072903D0067800248E422CD1012A0ED0002A02D0022A0FD013E041781400002921D100244279D209A2421CD109E000244278A242F5D188
:40B3C00016E000244279D209A24211D0002B06D002790024D206D20ED340DB0708D5054B01249D4204D043785C1B60424441E4B2200070BDFFFF0000F7B50F00060003F098
:40B4000097FB304B01220093802304001B0211003800FFF7B7FF002801D1002550E07B78042BFAD92300002581331D70FB7B9A06520FD1B2C81E01283ED820005B07DB0F38
:40B44000BC30037023007B331A70BA693D331A60042906D17B78052B03D9C623FA695B00E25022007B7A7C325B069B0F13702300012579331D70300001F0B4F822003B79B1
:40B4800096329B0913703000FFF718FF0421300003F0FCFC637D002B12D12300B9331A7818231A420CD12300C03470331978236830009B69984703E00629AED17434227069
:40B4C0002800FEBDFFFF0000932213B50B00002192005043034C00910A000059FFF752FF16BDC046B006002070B5060003F020FB0300A2331C780500002C01D100203EE07E
:40B500000300A4331B68002B01D0012037E009213000FDF7F3FC0028F7D1002E1AD1184B1A00FC32526D002AEFD15532FF329A5C002AEAD14422FF329B5C012BE5D0114B82
:40B540001A68114B1A42E0D1A023104ADB00D3589B05DAD4300003F0EBFAC023803002889B009A42D1D077352B78012BC6D0172CC4D0200008380400601E8441E0B270BDE4
:40B580000C050020A4000A400720000000000A40F8B5070003F0CCFA00210500380002F0DDFCA121354BC9005858354A932602405A50A02200243349B6007E43D2009950F2
:40B5C00038000E220021FDF753FC2F4B38009E192E4BF3181C7080239B00F3181C702C4BF3181C702B4BF3181C702B4BF3181C702A4BF3181C7082239B00F3181C70284BB3
:40B60000F3181C7081239B00F3181C808D239B00F3181C602B0081331C70013B1C700A3B1C70DC70013B1C7043331C60C6235B00EC502B00BC331C70453B1C702B331C7095
:40B6400002331C602A3B1C708233DC651C659C641C66C4235B00EC54FAF7B2FF114BF6182B0099333470013B5C701C711C70D6235B00EC540C4BDC55F8BDC04600000A40C4
:40B68000770EE9FF88F11600B00600200202000003020000060200000A020000070200000902000049020000AC06002010B50400FFF76EFF00212000FBF756F810BD0000F0
:40B6C000F8B5040003F034FA00210500200002F045FC932292006243214FBB18214A991800220A70204959180A70204959180A708221890059180A701D4959180A70812166
:40B70000890059180A801B4959180A708D2189005B181A602B00FC339A64DA65873B1A701A71944203D1144B4D33FF331C700A212000FDF7FDFB2B000026A4331E60083B3D
:40B740001E70D6235B00EE54A03363430B4AFB189B181E702000FAF733FF094B1E55F8BDB0060020030200000602000007020000090200000A0200000C0500204902000045
:40B78000AC06002070B50D00040003F0D1F9172D08D193239B0063430A4AD3180A4A9B1800221A70A230057009212000FDF7C0FB80212000490003F0BBFB0421200003F093
:40B7C000ABFB70BDB00600200A02000010B5040003F0AEF9030000219C33197093239B006343084A8430D318074A9B1819700378062B02D02000FAF7B7FF10212000FFF7B4
:40B80000C1FF10BDB00600200A02000070B5050003F08EF90300002677331E7004000A21280003F033FB31002800FAF79DFF28000221FFF7A7FF0423A434236070BD70B57B
:40B84000050003F075F903000026040075331E700E2231002800FDF70BFB230084331B78052B03D031002800FAF77EFF28000121FFF788FF0423A434236070BD70B50400A6
:40B8800003F056F9050081782000FAF7DFF80121200002F063FB20000E220021FDF7E8FA2B000022A4331A60012377352B701521200003F0EBFA70BD70B5040003F038F9D6
:40B8C000050000212000FAF74FFF2B0000226E331A70AD7C2000012D06D1FFF7E7FE2900200003F031FB01E0FFF7C8FF70BD000070B50D00040003F01BF9072D24D0082D55
:40B9000027D0022D40D1200003F012F905002000FFF7D6FE2B007033197850331B6820009B6998472B0001227D331A70174B18491A5593239B006343CB18164966355B185A
:40B940002A701A701A3217E003212000FFF71AFF1AE093239B0063430D4AD3180D4A9B181A78002A0DD00022C0301A7003680A491B6920009847094A09212000FFF7FAFCD1
:40B9800002E02000FFF798FF70BDC046EC0B0020B0060020450200006FB1000071020000F8B504000F0003F0C3F80300A1331D780600EDB2022F04D000D292E0052F77D9B2
:40B9C0008FE0484D48492B5D002B09D193228023920062439B008A18D218137801331370932380229B0063439200CB189B181A78032A10D9032276361A7033782000002B73
:40BA000002D0FFF759FF01E0FFF738FF01212000FAF7AAFE65E02B5D002B02D000232B5502E02000FFF74CFE002C02D00121295554E002F0A6FE052107002000FDF778FA33
:40BA400004212000FDF774FA07212000FDF770FAA121264BC9002933FF331C70244B254A5858254E02405A50A0222449D2009950234B38001C703300FC335C6533000527D8
:40BA80005533FF3345361C70FF3602F07EFE1D4B1422072137702000FDF76EFA0123184A39001370200002F009FA002819D0BDE71221200003F0EAF9002D07D076363378A9
:40BAC000002B03D12000FFF7F7FE0AE003212000FAF74AFE2000FFF7E7FB02212000FFF751FEF8BDAD060020B00600200403002000000A40770FEBFF0C05002088F0140059
:40BB00004F060020AD7E0000F0B593B0040003F00FF80300A2331B780500002B00D124E20600A4363368002B00D1BAE033689B0507D5030084331B78052B02D12000FFF77F
:40BB40007EFE3000F9F746F90290012801D006285CD1AC2702F015FE00217F006743CE4E0490F31934330393009120230A000398FFF708FC002810D02B00F61966331A7848
:40BB80003100012337315A400A702021303613405A01337A8B4313433372AC235B006343BD4AD3181A0034321278002A0DD12A003733663212781B789A4206D1049802F08B
:40BBC000E4FD2000FFF778FECFE19327BF006743B24E43220399B859FDF72EF9049802F0D4FDBA591378013B012B07D813792A009B09963213702000FFF760FB93239B002D
:40BC000063430C21F258200003F04EF9029B102B02D12000FFF713FE200002F089FF029B002B03D12000FFF7F1FD30E0029B012B22D1A230037820000E3B052B02D8FFF7FF
:40BC4000FEFD24E002F074FF932300269B006343924A9C30D318924A06709B181E702000302103F065F931002000FAF77DFD11212000FFF787FD0AE0029B092B07D1A2306E
:40BC80000378172B03D000212000FAF76DFD2B00A2331B78834A9B00D3189B6A0299200098472B0094331B78012B0ED92E00B4363368002B09D00B9307AA002311212000C0
:40BCC00002F0B2FE002800D130602B7C012B00D04BE1200002F02CFF93239B0063436F4A7149D3185D1829781700002940D07D300278002A3CD16D4A99180A78002A37D1D8
:40BD0000822080001B181878022826D8002803D108212000FDF70CF908212000FDF7EEF8002825D193239B0063431A00A932FF321D00BA185E4B0B21200002F075FE0028E9
:40BD400016D10121594A7B199A181170822292009B181A7852181A700AE01A70554B2A701B5D0A70012B03D10521200003F08EF8200002F0DDFE0600813633780500002BFD
:40BD800000D1F2E0030075331B78002B00D1ECE093239B006343444AFB189B181B78002B00D0E2E00300793304931B78002B00D0DBE003007D331B78002B00D1D5E00300B6
:40BDC000020094331B7880320292012B07D8030066331B78002B02D133701370C5E0029B1B78012B00D1C0E003212000FDF786F80390002800D0B8E02B00C0331B68200037
:40BE0000DB699847002803D1029B307018706CE03378022B1FD0032B30D0012B00D0A4E093239B006343244AFB189B181B78002B05D12A0082321370023333700BE0049BDB
:40BE40001B78002B20D12B2203212000FDF72AF90323337089E09322012692006243BB18D533FF331E701A000821144B200002F0DBFD002879D180352E7076E0049B1B78B2
:40BE8000DBB20493002B1BD06B466A461B7B127B3370029B1A7068E00C050020B00600200A020000ACF40000070200000902000069CB0000EC0B0020020200007DBF000060
:40BEC00093239B0063432A4AFB1803939B181B78059302F04BFD059B83420BD36B466A461B7C127C3370029B1A700521200002F0CDFF3AE00123039A2000D532FF321370C9
:40BF0000039AD932FF3213701B22039BE133FF331A7002F00DFE030095331978154A1300012903D97C3003785B031343932292006243BE1831003200E531FF31D5320B6071
:40BF4000FF320D4B0C21200002F06EFD00280CD1074B8035F6183378312201333370012303212B702000FDF79DF813B0F0BDC04602020000018000FF7DBF0000F0B58BB0FD
:40BF800005000E00170002F0D3FD03008133019304001878022811D1731E012B09D9002E09D12200823213780133DBB21370052B4DD903204BE0042E49D1FAE7032846D14B
:40BFC000042EF6D13F223B7A9343402BF1D139002800FFF711FA061E34D0270000237E373E78B200934207D019000D31FF31605803A958500433F5E7280002F0A1FD230011
:40C00000FC331B69039A53409B020ED12200113204A9FF320133B34208D201C9844601CA844509D10133DBB2F5E70023B34203D13A7800209A420AD028000B21FFF7A2FB61
:40C04000002004E02800052102F020FF3000002380342370019B18700BB0F0BDAC235B004343F7B51F4C1F00E3181A004432FF32019111780500012932D14533FF331E7808
:40C080000023033113700522FCF7F2FE032E08D8032307217343DB19E3181A7901320A401A71AC2252006A43A3184A33FF331E70B8235B006B430C49A120CB1800212933DE
:40C0C000FF331970094BC0001E58094931401950A0210848C9005850A358019928009847F7BDC0460C0500200403002000000A40770FEBFF88F0140010B5040002F018FD89
:40C10000A4300268094B1A4205D020001021FFF7A5FF012009E0AC2040006043044B1818FC30406D431E9841C0B210BD43C000000C050020F0B58BB00400089102F0F8FC30
:40C14000AC235B006343B5490500CB181A004532FF321278684600921A004C32FF3212782F0001921A004732FF321288943706926A46128B82811A004932FF32127856337E
:40C180000592069AFF33D20B04923F78069A07972F009537D2053F781B78D20D16000997002B28D0079B012B25D902230293059B002B08D0049B002B05D1049F1A3393424C
:40C1C0007F417B000293009B002B16D02B007D331B78002B0CD101225933FF336343CB184433FF331A7020212000FFF737FFA1E1099B012B01D803230293AC235B001900FA
:40C200006143864F79184331FF310878012802D10020087002906343FF185637FF373B78DBB2002B00D1C8E0059B002B2BD01A2A08D82B0098331B78002B03D1784B069972
:40C240000B430393039B1B04D90F049100210191D90F19D05B010BD41A26039B5B041B0F591C71438A4208D25E43961BB6B204E00026039B5B0A5B020393B01CF8F7CEFF69
:40C28000C3B2019300E0059E099B9901009B002B0BD12B006635673319782B7809025B0119430D00079B990129430322009B5B485A43AC235B006343D21882181579059A85
:40C2C0006D02D2031543C2184B32FF32127810331543019A1F18120315430D4320220021380003F010F80022019B05999B00DBB2914209D00499914206D06A469289F3B2EA
:40C300003A70120A7A700222D3180899DBB29A4205D008780131B8540132D2B2F7E76B4600229888059B93420BD0049B934208D1039B30001B041D43F8F770FF0122089F07
:40C3400080B2AC235B0063433449CB181D63B8235B0063433349CB1819002733FF33FC311A70009B4F6128310870022B05D180212D4AC90013680B431360009B9A002B4B5D
:40C38000D2582B4B1A60E0231B012B401A00009B0133190401231343264A0B431360264B0822DD606B469A56B8235B0063431D49CB182833FF331A7081E01A00009B002B32
:40C3C00007D12B00663567331A782B7812025B011A43AC200323009940004B4360430F4D1B18EB181E79019B76021B031E432B184B33FF33197840230B4333431343019AAF
:40C40000290096000022B24218D0089DAD580395039F15184D192F610432F4E70C0500200080FFFF04030020BC000A4044F50000C8000A40AC000A4000000A40AC204000B4
:40C4400060430A181363B822520062433A4D1030AA1815000918FC3569616846110000792531FF31087000212732FF321170009A022A05D180203149C0000A6802430A60FD
:40C48000009A91002E4A89582E4A1160E02212011A401100009A0132100401220A432A4902430A60294A2449D360B8226B46520062431B7A8A1828325BB2FF321370AC2564
:40C4C0006D00654302F05DF9214E012275192B004433FF3307001A702000FFF70DFE002825D12B004233FF331B78013B012B04D94A35FF352B78062B16D1009B013B012B00
:40C5000012D8AC235B006343F6185636FF363378002B02D0079B012B06D80E4B022204212000FCF729FD02E0200001F09BFD380002F02BF90BB0F0BD04030020BC000A40D5
:40C5400044F50000C8000A40AC000A4000000A400C050020AD7E000070B504000220002C1CD144200E4BFF301D5C3538FF38012D14D05620FF30185CA22040001954A52107
:40C5800049005A544C22FF329C54053A9C52023220009C542100FFF7CDFD200070BDC0460C05002002000220002A05D1032310005943024B59188A717047C0460C05002082
:40C5C00002000220002A09D10323594342230448FF334118C25410008A710A717047C0460C050020F8B5022300285BD102F0A0FA03002D4D943329681E782C4A2C4B0A4037
:40C600002C49012E07D90C682B4F3C430C6001245968214306E00F68284C3C400C6003245968A1435960822304000100077CDB01134367346631002F22D0070075373F78F9
:40C64000002F09D12778012F1AD1012E13D97D300078002814D00EE0012E05D906007D363678002E03D10BE00E78012E08D179300378002B01D1862300E08E23DB01134341
:40C6800041220F482B6003681B0C1B041A4323781C020B785B01234313430360094A0A4B1A6000231800F8BDBC000A40FF80FFFF00000A40E8000A4000001080FFFFEF7F63
:40C6C000C4000A4041004100C0000A40F0B58DB00400089102F02CFA93239B001A0083210F276243CB4E8900B21851180D78CA490390511809780491C8495118097805910F
:40C7000008A97F186946097D3970C5495118097809918521890051180968079184218900521812880692089A022A26D1059B013B012B02D9032D00D063E1039B94331B78F2
:40C74000012B0BD8039B66331B78012B00D158E1C4230121039A5B00D1545FE0039B7D331B78002BF4D0039B2000C0331B68DB699847002800D044E1EAE7089803380B2822
:40C7800000D9EAE102F0D2FD0C003A0046004E00E9018B00E901E901CD00E901E9011101032D03D11421200002F070FB3B78013B012B09D8002D07D1049B0D2B04D13A00A1
:40C7C0001321200002F070FB03212000F9F7CCFF93239B006343F618924BF6183288002A04D009212000FEF7C5FDB6E12000FEF75BFD17212000FEF7C5FFAEE16343F61888
:40C80000894B0021F6183378012B07D12000FEF7DDFFA2E1059B0121002BF7D02000F9F7A3FFE6E7634388218622F518F758872389006918098892009B00AA181278EB188B
:40C8400000911B6805993800FEF79CFD021E07D100900599754B3800FEF794FD011E12D093277F25BF00674317212000FEF78AFFF25904212000FEF74BFDF3595B79AB4323
:40C8800000D0A5E069E12000F9F76EFF664BED182B78022BBAD02000F7F7A0FC5DE102212000F9F761FF012D03D1049B11210F2B00D01021200002F0E9FA3B78013B012BB3
:40C8C00097D8002D95D1049B0D2B92D193239B006343F618514B0322F3181D7083239B00F3181A704C4B1821F3181D704D4BF3181D804B4BF3181D7085239B00F3181D6027
:40C9000084239B00F3181D8086239B00F3181D7087239B00F3181D6088239B00F618358068E709212000FCF703FB80212000490002F0FEFA932292006243B3181900A63136
:40C94000FF310978012900D153E700290ED1A533FF331B78002B00D14BE78932FF32B6180F2200962000FBF7A7FFF6E0032904D10D312000F7F726FBEFE0200002F0D8F8D0
:40C98000030094331B780500012B00D831E7030002229C331A70200019320921FEF7EAFC28001723A2300370D7E009212000FCF7BFFA80212000490002F0BAFA172280212B
:40C9C000039BC901A2331A70200002F0A5FAC4E00421200002F0ACFA2000F7F72FFBF159CB791A00AA430AD01A225B061B0F01335343CA88D205D20D934200D2ADE00421A5
:40CA0000E2E7032D00D9A8E0280002F0C7FA11171D80C046B00600200D0200000B0200000E020000120200000A020000100001003978049A2000FFF78FFD8EE0079B397811
:40CA4000049A0093099B8DE76B463E781D8B002C00D082E0424C23004433FF331B78012B7BD022005632069BFF321278D9055B04C90D1B0F002A27D0079A002A0CD101F09F
:40CA800080FE012305004434FF34002023701021FFF7E4FA28005EE0822252009142EED8069AD802550A6D022E4A0D432A4002437B20151C120A8243802A05D1002B03D08D
:40CAC000663A5A439142DAD922004532FF32167022006E464B32367CFF321670220000204C32FF326D0A10706D02DA021D4B294319400B00134322004732FF321380012323
:40CB00004934FF3423700799FFF714FB25E001212000FFF755FD02212000FFF751FD002C1BD10F4B1D004435FF352A78012A14D006264533FF331E7001F023FE0123070069
:40CB40002B702000FFF7D8FA002803D13100200001F0B4F9380001F018FE0DB0F0BDC0460C050020FF87FFFFF8B50F001500040001F0DEFF6E22060008212000AD78FCF749
:40CB800091FA042F2CD1EB1E1E4F012B01D9102D1DD108212000FCF7CBF993239B006343194A8220FB189918002280001B180A701A70042D06D1813632700521200002F0E1
:40CBC00065F904E0032D02D101230B7018E093239B005C430D4B3F19FF1800233B700FE0032F04D108212000FCF7A2F908E093239B005C43034B1C19044BE41800232370AB
:40CC0000F8BDC046B00600200702000009020000704710B5472902D1BA31FF3103E0482903D18021C900FDF7A9FD10BD10B5FDF7A5FD10BD70B504000D0001F08FFE9430DC
:40CC400003780422012B00D90C32702363430449C8180833027359182000A84770BDC04688040020F0B587B00E000700059201F075FE94300378C54A029370237B43D31850
:40CC80001900002080242D3108703189C048240208401100A04200D0F1E0B2681A61727A3B335206920F1878D4B2031CA04200D9131CDAB2019270227A438A1811003B3169
:40CCC0000B70130001212C3319703F23107C03408020404203431374AE4BD85DAB4B002803D00298884200D8BAE07278012A00D0B8E0307AC006C00E0138052800D9B1E0FC
:40CD000002F04CF9034E75B0B0A8FF2271891202914200D0A6E0A04AD15D002900D1A1E0702078431A182C3211709C4ABD00AA58964E94468A000292002264461518A45831
:40CD4000AD192C61029C0432A242F6D1019A002A76D170327A43B6187069F27D904D92062840904D520FD60628403043360E182E00D1019A07263240D20628401043120E46
:40CD8000283A54425441221D8A4204D27021794359182C310A7070227A439A1850614FE0FF227189120291425CD17F4AD25D002A58D07020784319182C310A707B49BD0042
:40CDC0006958724E8C4600219200644645186458AD1904312C619142F7D170227A43B6183F22317C0A4040210A4332743AE070497A00895C042935D96E4AB80080587589CB
:40CE0000C6880278AE420DD170257D43043A591992102C310A705D4CD2B2013292000021A44605E080188A1AD1B20029E8D119E004318A4204D04E1944586644F460F7E7AE
:40CE400070227A4399183F22087C0240402002430A7407E070227A439A182D32012100E02D32117070227A439B1803226021019C144062015C7C8C4314435C749CE24E4A5F
:40CE8000D37A917A1B020B4311D172893F4D9A4200D0F1E170237B43B168ED18296118216B7C8B4308390B436B742C3582E272899A42EAD13200317A0C320492CA06D20EBB
:40CEC000039272683D4C55044A0918210192627A207A8A4310390A436272019A1731014052010A436D0F2272039A013DAD00501EEDB263811328C8D802F00EFA14002100BE
:40CF000068009A00AC00C600E1000201230140014F01C7FF5D018101A102C7FFA102C7FF8A019301002D0CD1254B1B78E360002B00D086E22F3323610335313B84E1002D7E
:40CF400007D01822637A01259343083A1343637278E12200E0230C3203CB03C2194B21001B785B0706D4184B59680902090CC9016131FF3120000822143002F0BBF9002390
:40CF80000725E3612362023B5EE1C04688040020C080FFFFEC0B0020B2020020B4020020FFFF7FFCFFFFFFC7B8020020BC020020C0020020C4020020001900000009002050
:40CFC0006C00002094060020C0FF0000042DB8D1337B532BB5D1D14B9B6C2361D04B1A78D04BD1B261611B781B020B431A006361CD4B1B781B041343CC4A63611278120694
:40D0000013436361CA4B1A78CA4BD1B2A1611B781B020B431A00A361C74B1B781B041343C64AA361127812061343A36100230BE1042D86D1337B522B83D1C14A03210020EA
:40D0400001F004FD033D0C23002800D0FCE0BD4B186009E1042D00D073E7327B09234A2A00D0B4E10321E33318780B00084000D0ADE1B34A01F0EAFC0C23002800D0A6E107
:40D08000B14AB04B1A60EFE0042D00D059E7337B0222611D502B08D1CB7F033D934300D0D1E10634CA77E577CEE0C87F0323104200D1F0E10023A21DCB77D377EBE1019BAE
:40D0C0005E1EF3B2052B00D93BE7019B062B03D0182D00D035E702E0082D00D031E7182070439A4BC0B2083018182A00049902F001F90122B24096490B8893430B80B3E03C
:40D10000042D00D01DE7934B1B7A002B00D018E7337B462B00D014E78D4A1388002B0DD1B37B717B1B020B433F2111808A4A1BB2934203D1894A13781D43157001250523C7
:40D1400082E0002D00D0FCE6019B591ECBB2052B00D9F6E6182359430198C9B20822062800D01A002000794B083159180C3002F0C1F8019B0725062B64D166E1042D00D0E1
:40D18000DFE6337B462B00D0DBE60534E27F3F3B002A00D01BE1073319E1042D00D0D0E66F4B347B1B78A34200D10FE1012C00D10FE107230BE1082D00D0C2E6737B317B18
:40D1C000B07B1B020B4300041A000300F07B134300061843737C357CB17C1B022B4309041A000B00F17C1343090619435D4B42189A4200D9A5E6FBF729FE207321E1002D81
:40D2000000D09EE6FBF7DAFF2561E060033519E0002D00D095E6EC23E5601B780235237310E0019D013DEBB2012B00D90FE1FBF7C5FF2B01C0330C3419181022200002F0C4
:40D2400059F8052502235B421F2047490A7A8243039802430A729A1C00D1FBE0424A01350233EDB2D360F5E070237B433F4AD31802222D331A709FE0380001F06FFB039085
:40D280003800F4F727FF4378DB0600D48AE0384B72899A4200D085E0334CB368A360A023237273685B045B0F012B75D1314AD25D0192002A70D1727A317A5206520C0A436F
:40D2C0002D498A4224D004DC2C498A420AD02C4903E02C498A4259D02B498A425CD150222272CAE0039B3800C0331B681B6C98470A2101F05DFE6B461B7980B223736B4637
:40D3000060730005000FA0731B79E3730223B4E0019BE36004232373023BAEE0FCF0FF0F78F1FF0F79F1FF0F7AF1FF0F7BF1FF0F7CF1FF0F7DF1FF0F7EF1FF0F7FF1FF0F1B
:40D34000918C00008C0600204C4200008009002086000020000A0020FF010000940600206C000020FFFF00000009002088040020C6050000EC0B0020030C000003060000C4
:40D38000030B0000030E000003100000019BE360302323732E3B70E070237B43ED182D35022308E070237B43029AED182D350323012A00D801232B7070237B433A491033A2
:40D3C00059183800059B984707B0F0BD002301253AE7364B9A68197B120A0906114326D05A681002000CC201100080300192421894462F4A94451AD81A681E79120A3606CC
:40D400003243904213D8944511D91E78FBF71EFD86420CD101988130FF30FBF709FF002805D1244B1A78AA431A702500FEE50421204A012513780B431370062304E7012573
:40D4400001E00225FEE60323FEE60325FAE601250723F9E67021002279431348164E43182C331D70AD00340008348B181459C31804321C61AA42F6D19EE770227A43AD1803
:40D480002A002C321370A2682A61022B00D093E7E3686B6190E71F21227A01258A4319390A432272DAE6C04688040020C0FF0000FFFF0000940600200009002070B504008A
:40D4C0000D0001F04BFA02007D32127803000320012A05D0D979090901402000FAF76AF970236343034AD1180833087399182000A84770BD8804002070B504000D0001F08A
:40D500002DFA702262430C498A18433213780E000122002B06D1C179033319402000FAF749F9020070236343F11808330A732000F118A84770BDC04688040020F7B5002088
:40D5400001F0F6FAAD4AAE4B0190D15817000093002900D1ECE1D3589B050CD594220020A84B5200985408211B6898478822A0239200DB00FA50009BFA5880231A4207D08A
:40D58000A0229E49D2008B5001219E4AA833D1549D4A9A4BBA58120624D5A2222A21D2009858FF31974AC00501D5002314E0012050549521DB6D4900DB01DB0D03339B10D7
:40D5C000DBB25354535C412B01D9412353542C210023FF31535401315354C022A2235200DB00FA508024009B2403FB58234205D0F7F728FEA023814ADB00D450009A7F4BC1
:40D60000BA5852016DD5A022D2009E5894467D4C32071CD530223240102A18D11932FF32A15C012913D1002080257849A0540A682D032A430A60A121C9005D58744A2A4023
:40D640005A506146734A5A502368032198472A25FF35F3073AD520231E4037D1A1220933FF33E654D200B9586B4B0B40BB508022A0235201DB00FA50684B019A1B68943261
:40D680009B065B0F013B2371F96DA1601378012B02D8634B0B40A360637A5B065B0F6371DAB2237AD9069B06DB0FC90EA171E371635D002B04D15B495B48FBF7BDFB01E0BD
:40D6C000F7F7C0FD0621002023689847A023574ADB00FA500023E0226355A2239200DB00FA508024009BE400FB58234208D0454B07211B6800209847A023404ADB00D450B3
:40D700008024009B6402FB58234208D03D4B07211B6800209847A023384ADB00D4508021009A4901BA58354B0A420DD0A120C0001C58394A22401A50A022D2009950314BC1
:40D7400001211B68002098470224009BFB58234208D02C4B0B211B6800209847A023274ADB00D4508024009BE402FB58234D23420ED00021080000F031FC002805D1A1222A
:40D78000D200A9582A4B0B40AB50A023DB00FC50009B1A4CFB589B0461D5942200202821184B5200FF3198545A5C1D0052B20191824209DAA121C9006558154A2A40625005
:40D7C0001B680221984745E0019BEB5C002B3BD0A0238022DB005203E2500520F8F7C9FF8022144E12033368134225D0A1228021D200A35849030B43A35025E000000A40B8
:40D800000C050000040300201C050000AC000A40771FFFFF88E00000FFEFFFFFA4000A40EF7FFFFF60000A40100300207F000804FFFFFBFFC4000A400520F8F79AFF80229A
:40D840003368120313433360019B019AEB5C013B5BB2AB548022A0239201DB00FA508025009B6D03FB58C24C2B4211D00520F8F780FF8021BF4A090313680B431360A12285
:40D88000D200A158BC4B0B40A350A023DB00E550009BB74CFA58C0231B021A421AD0D022A0231202DB00E250A1228025D200A3586D012B43A3500A20F8F75BFFAF4B1A6886
:40D8C000AF4B1A4201D1AF4BE5500021AE4B08001B689847009BA64CFB58DB0511D594220020A94B5200985405211B689847A122D200A158A54B0B40A350A023A44ADB00CF
:40D90000E250009A9A4BBA58920311D594220020A1249D4952008854E4001D599B4A2A401A51A0229A4CD2009C500B6804219847984C8F4B3A59002A78D01A59D20132D5F9
:40D94000D02252009B581B011B0F042B03D10020F9F702F922E0AC218B4B49005A5C0F2A07D8501C58548C499A18496F4932FF321170AC2149005A5C0F2A08D8501C5854DF
:40D9800085499A18496F4932FF32090A1170FC335B6B002B02D04021002098478022A4235204DB00FA5080233A599B041A4203D0A4226F49D2008B503B59DB0414D5A42367
:40D9C0006B4ADB00D258754B80211A4200D049006D4BFC335B6B002B01D0002098478022A4235201DB00FA5080233A599B011A4203D0A4225E49D2008B5080253B596D034A
:40DA00002B420AD0604BFC335B6B002B02D0202100209847A423DB00FD5080233A599B031A4203D0A4225249D2008B505C4C50493B59002B24D011230A591A421FD0A62224
:40DA4000D2008B5001227033FF33C8581043C850F8581040FCD1C0231F21454A5B00D558494B6A0AFC33AD0B9E6B0A402940511A8E199E635B6B002B01D0102198473B59AB
:40DA8000484C3B4A3B595B0000D4ADE01359464BD158C90711D545497F205158444D8C4666463040C0038446515942480140604601435151002240490A70FA582C483F49CB
:40DAC000D2050FD5394A8558394AED0A9446825816003B4A15403B4A324015436246855000220A70C020A8220006D200B85036480200B63215780200B732127812022A4310
:40DB000012182D480078002803D10878C0B2002860D00978002909D00120F9588143F950F958FF300143F950108B08E0F858274901400120F950F9580143F950108F1823D3
:40DB40005843013880B2F7F713FAC022A8231206DB00FA50A9228021D200BB58C9050B430121BB501A4ABB580B43BB503CE0C04600000A40C4000A40FFFFEFFFA4000A40FC
:40DB8000072000000405000004030020FFFEFDFF000102002C050000FC000A40000001103C0500004C0500004C20000054200000F4080000FF7FC0FF790600207A060020A0
:40DBC000E07F00001F80FFFF00190000FFFEFFFF502000000121134AD050134B1970134B1B68002B00D0984780233A59DB011A4209D0A8220B49D2008B500D4B1B68002B4C
:40DC000001D00020984720233A591A4209D0A8220449D2008B50054B5B68002B01D000209847F7BD00000A40780600200C0A0020FC040020F7B5C524060000F0A2FDC02239
:40DC4000154DE4002B59920113432B5107001420F8F78FFD01213000F7F764F8B8235B005E430E4B01909E19FE36368B0C4B2A59142013402B51F8F77CFD380000F085FDC7
:40DC80005020019BB6B25E43360A7043D22101F019FA80B2FEBDC04600000A4004030020FFCFFFFFF0B585B0070000F06AFDF022C52102902020384CD200A358C9005B00BE
:40DCC0005B08A35063580426034363507821A35800258B4360390B43A350403AA3582F4912300B40C02109030B43A350F8F741FD2A4B039301213800F7F714F8013E2D18D7
:40DD0000F6B20A20F8F735FD002EF3D1B8235B007B43234AAD08D318FE3301931B8BE8B25843204B000A7D36984214D9E822D200A358039932200B40C02149020B43A350F1
:40DD4000F8F717FD01213800F6F7ECFF019B5A3E1B8B5843000AFA25134BAD001978684301F026F9310001F023F9F0227821D200A35805008B43A350593AFF3AA3585839A5
:40DD80008B43A3500A20F8F7F4FC029800F0FDFCA8B205B0F0BDC04600000A40FF7FF0FF040300203A07000084000020F7B50600F7F7E8F801213000F6F7B4FFB8235B00E9
:40DDC00073431F4A1F4FD318FE3300931B8B43431C003B785C431C4B640AA4B29C422CD800F0CFFCC5230822184D0190DB00EB580A201343C522D200AB500A233B70F8F764
:40DE0000B8FC01213000F6F78DFF009B08221B8B43431C003B780A205C43C523DB00EB58640A9343C522D200AB5019233B70F8F7A0FC0198A4B200F0A8FC2000FEBDC04606
:40DE400004030020880000202723000000000A40F8B5040000F095FC8022134E134D920073590700134373511420F8F782FC01212000F6F757FFB8235B0063430C4AD318E8
:40DE8000FE331C8B0B4B44431B7872595C430A4B142013407351640AF8F76BFCA4B2380000F073FC2000F8BD00000A40CC0800000403002088000020FFFDFFFF70B50C0072
:40DEC00005290CD102221C4DFF322B68080013432B60F8F74EFC2A68184B13402B60A022A121174B1748D2009850C9005A5802435A50154BA200D258144B1A60052C07D05B
:40DF00008021134AC902136800200B43136011E00A24104B104E1A681D00324206D0013C0A20E4B2F8F725FC002CF2D12B680F203342E5D070BDC046DC000A40FEFEFFFFC0
:40DF400000000A400001020044F50000CC000A40C4000A40A4000A4007200000A32010B5184BC0001C58184A22401A50A2229938FF38D200985000290AD11449144A0868E0
:40DF800002400A60A121C9005858124A024011E0012910D10D490E4A086802408020C00102430A60A121C90058580A4A02408020800002435A50A0220749D20000209950A3
:40DFC00010BDC04600000A407FFEFFFFBC000A40FF80FFFFFFF9F6FB00060904F0B51E4B1E4C1A68B8235B004343E3182533FF331B78002B01D100202DE0002906D11F23D0
:40E0000008241340072B03D8210001E010240021B8220B0052005043104A10180A19934218DA050006002635FF352A78FC367669920097591A1D0A4E920097512A78013D0F
:40E040000132D2B26A706A782D789542D3D90133DBB2E3E70120F0BDA0000A400403002000000A40F7B5A125414BED005959414A04000A405A51A0223F49D2009950B82251
:40E0800052004243944601923C4A1E00944460462830FF300278394F52B2002A06DA8020374980015A5802435A505EE0354A12681100354A0A400FD002780021013A52B257
:40E0C000027080205A59400102435A51019B2B4A20009B58984748E063462633FF331A7001212000FFF77AFF002804D080227359D20213437351A122D200B35823481C49C8
:40E100000343B350B8235B001A006243BA182732FF3212780220012A02D14A68024301E04A6882436343FB184A6028331849FF330A681B78002B03D080231B031A4301E0F9
:40E14000144B1A4080239B021A43B8235B005C433F193B0000202933FF3328371870FF373B78013B5BB23B700A600120FEBDC04600000A40FFEFFFFF98F01400040300202A
:40E1800004050000A4000A400120000088E00000C4000A40FFFFF7FF0221024A53688B435360704700000A4070B50D0000F0D6FBC0221D4CD200A1581C4B0B4010210B43F7
:40E1C000A350002D0AD08B30037819489B001B5CA15858025B0103430B43A350AA239B00E158144A0A200A40E250E25812490E4D0A43E250F8F7BDFAAE2370229B00E2505C
:40E20000B02260219200A3580B43A350AD239B00E258A0235B011A4205D0AF229200AB5840390B43AB5070BD00000A400FF0FFFF1CF40000E8A3FFFF05140000012270B532
:40E240000600214C214D3220635993436351F8F790FA3000F3F74CFF0230C37F002B09D0802280216359C9041343194A6351A3580B43A3500722174E0120A3599343BC22FB
:40E2800012061343A822A351134BE250F8F771FA8022FF21A359D2011343104AA351A35832208B43FE390B43A350A1580C4B0B40802189030B43A350F8F75BFA0222635953
:40E2C0009343635170BDC04600000A40EC08000078200000DC080000E4080000E8080000FFFF00FFF0B585B00090F3F701FF060000F047FA0290F8F731FF264C264D002885
:40E300003FDA12226359254F134363511823308B80265843013880B2F6F72AFE012200211F4BF605E2501F4BE15063591E499B025B0E6350A8211D4BC9006650E058024320
:40E34000E25001930391039BE35833420AD1013F002F03D10098F8F759FC03E00120F8F708FAF0E76259124B134063518022A823D205DB00E2500122019BE3589343019A54
:40E38000A35062590B4B13406351029800F0FDF905B0F0BD00000A40F4080000A08601004C2000005C20000058200000502000001F00C0FF0500C0FFF7B5B123B0215B4C99
:40E3C0009B008900E258635893436350AE239B00E2503D33FF33E258002A00D10FE10825E3582B4200D1B0E0514F3B680093002B53D0FC26B600A3590020AB43A351FA23C9
:40E400009B00E550009B984700233B60FC230121DB00E2588A438021E250E25809060A43E250444A1268002A00D18EE0D622D200A1589446404AE8200A403979C000A940D1
:40E44000114300911F2122588A4301927A791140019A11436246215000990A20A1500121E2580A43E250E2588A40CA40E250F8F780F9E321890063589B0A9B026350BB79A9
:40E48000625858010523134303436350FA239B00E550A3591D43A55157E0E326B600A3595B079B0F022B26D1FC229200A358AB43A350FA239B00E550FB79591E012904D807
:40E4C0001C4B00981B6898473FE0032B3DD10121A3598B43A351A35905318B4305310B43A351A3580E311D43A5503A7A134B0098FAF742FD29E0FA239B00E55019210098D7
:40E50000FAF7FCFC00281BD019210098FAF710FDFA2301229B00E550A3599343A351A3590D329343093A1343A3510EE000000A40140A002068060020FF00FFFF7D640000B9
:40E54000FC229200A358AB43A350FD2201219200A0580A00764D774BEE68B24002420CD0FC26B600985990439851FA2080001A502B69002B01D000209847FD229200A1588B
:40E5800001226C4B11420ED0FC208000195891431950FA2189005A50674B1B68002B02D0002108009847FD229200A1581022614B11420ED0F821FA208900800059581A506E
:40E5C0005E4BFC33DB6E002B03D0C903C90F00209847FD229200A1582022564B11420ED0F821FA208900800059581A50534BFC339B6E002B03D08903C90F002098478A2261
:40E60000D200A15802224B4B11420CD04C481958914319504B495A504B4B1B68002B02D00121002098478A22D200A1580422414B11420CD0424819589143195041495A50AB
:40E64000424B1B68002B02D000210800984794228821D200A2584904364B0A4206D03C483C4A1D582A401A503B4A99509422D200A15801222F4B11420DD035481958914399
:40E68000195035495A502D4BFC335B6B002B02D00221002098479422D200A1580222254B11420DD02A481958914319502A495A50224BFC335B6B002B02D004210020984738
:40E6C0000422264D1B4B615911420BD0244819589143195023495A50154B5B69002B01D000209847012263591248134211D01D4BC250124BFC335B6E002B0AD01A494658A0
:40E700000021164203D019494158D140114000209847102362591A4208D0124A05498B50034B9B69002B01D000209847F7BDC046140A002000000A40780400200403002038
:40E740004C0400004404000084060020800600209C040000FFFFEFFE9404000048200000442000003C200000F4080000382000000230800803D00138FDD1C046C046C0466C
:40E780007047EFF3108072B6704780F310887047F8B505000220002D55D1002953D02A4C2A4A2300CC331A602300C03319602800FAF71CFB010066222031200000F09AFD56
:40E7C0002800FAF713FBC189214E00290CD0FAF715FB07002800FAF709FB818918227918300000F087FD03E01822300000F08BFD0020FAF7FBFA418A164D00290CD0FAF7A7
:40E80000FDFA06000020FAF7F1FA018A15227118280000F06FFD03E01522280000F073FD2378022B00D063700020F9F777FB0020F7F7E4FE2300012288331A70D4230020EF
:40E84000054A5B00E250F8BD380A0020080B0020A40B0020C80B00200789341410B50222002813D10A4B19008831097800290DD0DC7C0A32002C09D11A008932147001221F
:40E8800087331A702000F7F7FBFC2200100010BD380A002010B504000220002C08D1054B88331B78002B03D02000FCF7E7FF200010BDC046380A002010B50A4B87331B786D
:40E8C000002B01D101200BE00020F7F733FC002801D0002004E0FCF707FE0028F2D0F8E710BDC046380A002010B5FFF7E5FF041E07D0054B87331B78002B02D00020F7F79F
:40E900000FF9200010BDC046380A002010B5F7F7BFF8012010BD000070B505000224002817D10D4B1A0087321478002C06D0F7F757FA2800FDF7E8F82C000AE089331A786A
:40E94000012A06D120001C70F7F780FC2000FCF7ADFE200070BDC046380A0020DA235B005843014BC0187047380A0020014B98787047C0468A000020014B18787047C04680
:40E98000300A0020014B58887047C046300A002070B5050014000720002D40D1204A1000873005780B20002D39D0150072352D78002D34D0100085300078002804D110002C
:40E9C000A4300068002802D00F20052927D11000A2300078172806D0082801D1002902D00B2005291BD110000125853005701000843001701100C4310B60C42300215B0072
:40EA0000D1548C4205D0CC32106821002C2200F071FC802103488900FAF701FA002070BD380A0020DC0A002010B504000720002C08D105489C3004780F20002C02D12000DE
:40EA4000FFF7A6FF10BDC046380A0020030070B50720002B18D10D4B1800873004780B20002C11D01D0086352C780430002C0BD11800C8338A3001701A6005488021FAF739
:40EA8000CEF9012320002B7070BDC046380A0020E00A002070B50224002844D14B005B0F0A34002B3FD0214A15007E352D78AB4239D841339B00D318DD79AD09032D20D15F
:40EAC000150094352D78012D06D8C03213683A211B680200984726E01A794D065206520E6D0EAA421FDB0525DA880903D205120E6A43490D8A4216DB5B795D43A94212DBBB
:40EB00000AE09B880A0E9B0522409B0D002A05D00903890D8B4206DB040004E08905890D8B4200DB1400200070BDC046380A0020DA235B005843014BC0187047380A00200A
:40EB4000F0B5914B914A1D88DA235B004343D3181900793109788FB0019000291CD06020B833197896250840402800D1FA25DA23019C5B006343D3181C007B3424786D00F1
:40EB8000042C09D1B8339B783F2B02D9002800D15A25C906C9170D40DA2301995B004B43D31867331B78002B01D1FA256D006B00052128000B9300F0FBF983B209937F23C5
:40EBC000099A01991A400C923633019AFF335A43089217006E4A6D4B51430022039205920492089A2037FF189B18029309330A910D930D9B049A1B789A4200D390E0029B10
:40EC0000049A9B7A13410122134200D183E00A9B089ADB199C58FA783B6892091B030692029A9B0D07939432BB7812789B069B0F012A08D9069A1E00032A51D8100000F0C0
:40EC4000ADF90B2B3943069AA4009207A4081443120EC02AEED15EE0A005800DA84206DDAB05A40A9B0DA4021C43002636E04949079A0C409202484914430C401A05144352
:40EC80001E00002A2CD06E236421584300F01AFAA84225D9002623E007990B9A1E004A43A105890D8A421BD29205A40A920DA402144313E0A205920D1E00954210DAAB05BC
:40ECC000A40A9B0DA40208E01E00099B6206520E934205D27F239C430C9B1C43012303932C4A079B14409B021C432B4B36051C403443069BA4009B07A4081C436D23019AB0
:40ED00005343059A9B184233204A9B00D3185C60059B01330593049B04370133049368E70820029B02999B7A0931FF31DB09DA00CB7983431343CB71029B94331A78029B9E
:40ED4000FC33012A04D81969144A0A401A6107E01869134A02401A610122CB791343CB71DA23019A5B005343084A6946D3181A00097D7E3211706A460120127B8A33FF33AA
:40ED80001A700FB0F0BDC0468A000020380A00204CFEFFFFFF03F0FFFFFFCFFFFFFF3FFEFFFF3FFFDA235B00434310B5034AD318FC33196DFFF76EFE10BDC046380A0020A8
:40EDC00002207047DA235B005843054B1B1894331A780C20012A02D9012200201A707047380A002010B5FDF7DDFB10BD10B504000220002C03D12000FCF758FC200010BDB6
:40EE00000223002803D1034BB4331960030018007047C046380A00200223002803D1034B9B331970030018007047C046380A002010B504000220002C03D12000FCF75AFA77
:40EE4000200010BD0223002804D10122024BA1331A70030018007047380A002003000220002B03D11800024AA13213707047C046380A00200223002803D1034B9C331970BD
:40EE8000030018007047C046380A0020DA235B00434310B5034AD318C0331B6800221B68984710BD380A0020DA235B00434310B5034CE318C0331B681B68984710BDC0467C
:40EEC000380A0020002310B51A000521FFF7ACFD10BD000070B5DA2464004443084B00211C199B3405002678F7F7F2FB2378B34204D0802128004905FFF782FF70BDC046F3
:40EF0000380A0020DA235B005843024B1818BE3001807047380A0020DA235B00584310B5024B1818A430F9F77AFF10BD380A0020DA235B00584310B5024B1818A430F9F7DD
:40EF400061FF10BD380A0020DA235B00584310B5024BA830C018F9F762FF10BD380A0020DA235B00584310B5024BA830C018F9F749FF10BD380A0020014B18180079704705
:40EF8000300A0020014B181801717047300A0020014B181841717047300A002002B4714649084900095C49008E4402BC7047C046002243088B4274D303098B425FD3030A1E
:40EFC0008B4244D3030B8B4228D3030C8B420DD3FF22090212BA030C8B4202D31212090265D0030B8B4219D300E0090AC30B8B4201D3CB03C01A5241830B8B4201D38B036D
:40F00000C01A5241430B8B4201D34B03C01A5241030B8B4201D30B03C01A5241C30A8B4201D3CB02C01A5241830A8B4201D38B02C01A5241430A8B4201D34B02C01A524117
:40F04000030A8B4201D30B02C01A5241CDD2C3098B4201D3CB01C01A524183098B4201D38B01C01A524143098B4201D34B01C01A524103098B4201D30B01C01A5241C30866
:40F080008B4201D3CB00C01A524183088B4201D38B00C01A524143088B4201D34B00C01A5241411A00D20146524110467047FFE701B5002000F0F0F802BDC0460029F7D052
:40F0C00076E7704703460B437FD4002243088B4274D303098B425FD3030A8B4244D3030B8B4228D3030C8B420DD3FF22090212BA030C8B4202D31212090265D0030B8B421B
:40F1000019D300E0090AC30B8B4201D3CB03C01A5241830B8B4201D38B03C01A5241430B8B4201D34B03C01A5241030B8B4201D30B03C01A5241C30A8B4201D3CB02C01A33
:40F140005241830A8B4201D38B02C01A5241430A8B4201D34B02C01A5241030A8B4201D30B02C01A5241CDD2C3098B4201D3CB01C01A524183098B4201D38B01C01A524199
:40F1800043098B4201D34B01C01A524103098B4201D30B01C01A5241C3088B4201D3CB00C01A524183088B4201D38B00C01A524143088B4201D34B00C01A5241411A00D2EA
:40F1C00001465241104670475DE0CA0F00D04942031000D34042534000229C4603098B422DD3030A8B4212D3FC22890112BA030A8B420CD3890192118B4208D389019211F1
:40F200008B4204D389013AD0921100E08909C3098B4201D3CB01C01A524183098B4201D38B01C01A524143098B4201D34B01C01A524103098B4201D30B01C01A5241C3081E
:40F240008B4201D3CB00C01A524183088B4201D38B00C01A5241D9D243088B4201D34B00C01A5241411A00D20146634652415B10104601D34042002B00D549427047634690
:40F280005B1000D3404201B5002000F005F802BD0029F8D016E770477047C046014B18687047C046F00000200E4B70B500251E000D4CE41AA410A54204D0AB00F3589847B5
:40F2C0000135F8E700F04EF9084B00251E00084CE41AA410A54204D0AB00F35898470135F8E770BD70F5000070F5000070F5000078F50000002310B59A4203D0CC5CC454E1
:40F300000133F9E710BD03008218934202D019700133FAE77047000003B47146490840004900095E49008E4403BC704703B47146490840004900095A49008E4403BC7047D7
:40F34000000000008A8C909C9492BCBAB6BEB800FD250000118C0000D573000085760000857C0000C11F0000AD1D0000BD1D0000151F0000DD2400003D240000DD1E00006B
:40F38000F9D4000035CC0000BDD4000065CC00000D1F0000AD73000088132823803E2C01010000001412100E0D0C09060302141211100C090705030214130F0B070504036D
:40F3C000020114130F0C0705030201011412100F0D0C0A060402141311100D0A070504031513110C0907060504031514100C08060403020204000000A5A60000EDAC000022
:40F4000099AF0000A1A60000A5A6000051AC000049AB0000F9A80000A1A700000006000001060000040700000003050700010200295800008D63000099580000E55900004E
:40F44000A94C0000A95C0000A95C0000A55500005A000000960000002C010000645F645F645F645F645F645F645F645F645F645F645F645F645F645F645F645F0C000E002C
:40F480000F01100210030F040F0600005A00000055000000500000000A000000150000001F0000006400D200F000000000100000002000000000000000000000000000005C
:40F4C00000000000000000000000000000010000000001006DB10000A1B90000F1B80000B9990000CDA3000005990000D19A00002D9E00001D990000C99D000079A100001D
:40F5000039A5000091A40000D9990000ED9F00003DA20000199D0000D59C000019410000CD3D0000A59B0000A53E0000353E0000E9440000CDC600000000000000000000FA
:40F540000000000018E30800181B0300D860030038670300389B080093730E008C0F0E0043000000F8B5C046F8BC08BC9E467047491D0000BD690000F8B5C046F8BC08BC1D
:40F580009E467047211D000098F500006800002090000000F80A00000000000003000000FFFF00004E6F7420537570706F7274656400000032003F0019002C0114000000E8
:40F5C000000000000000000000000000000000000000000000000000000000000000000060F5000000000000000000000000000000000000000000000000000000000000B6
:40F60000000000000000000000000000000000000000000000000000000000000000000090000020000000000000000000000000000000000000000000000000000000001A
:40F64000000000000000000000000000000000000000000000000000000000000000000000000000000000000000000000000000000000000000000000000000000000008A
:40F68000000000000000000000000000000000000000000000000000000000000000000000000000000000000000000000000000000000000000000000000000000000004A
:40F6C000000000000000000000000000000000000000000000000000000000000000000000000000000000000000000000000000000000000000000000000000000000000A
:40F7000000000000000000000000000000000000000000000000000000000000000000000000000000000000000000000000000000000000000000000000000000000000C9
:40FFC000F5011D00002F00000080DE000000000000000000FFFF594302000000000000000000000000000000000000000000000000000000000000000000000000000000C5
:0200000490303A
:020000007399F2
:0200000490402A
:40000000FFFFFFFFFFFF00000000000000000000000000000000000000000000000000000000000000000000000000000000000000000000000000000000000000000000C6
:0200000490501A
:0C00000000022B0711BB00012B56855499
:0200000490600A
:0100000001FE
:00000001FF
